:020000040000FA
:10000000B031172BFF3F27004C08003A03193D2859
:10001000F1017108073C031C2A282900A31B13289F
:1000200021008D13152821008D170630FD00FD0BD2
:10003000172800000D170630FD00FD0B1D280000DD
:100040000D130630FD00FD0B232800002900A33509
:10005000F10A092821008D170630FD00FD0B2E281E
:1000600000000D170630FD00FD0B342800000D13B5
:100070000630FD00FD0B3A280000080027004C0860
:10008000003A03195C2821000D170630FD00FD0B16
:10009000472800008D170630FD00FD0B4D2800009D
:1000A0008D130630FD00FD0B532800000D130630A4
:1000B000FD00FD0B59280000080027004708280014
:1000C0006F072900A2003E20270045082900A30051
:1000D00003202900A301032028006E08B03E290058
:1000E000A3000320290022080F3C031C7B282208C0
:1000F000A000A1018C282208F200F236F236F23676
:10010000F2367208A1007208F000F035F035F035D3
:10011000F03570082202A0002008A3000320290067
:100120002108103EA30003203E2027004508290097
:10013000A300032040302900A30003200800200072
:10014000F801F9011030FC00710DF80DF90D74087B
:10015000F8027508031C750FF9020318B628740815
:10016000F80775080318750FF9070310F00DF10D66
:10017000FC0BA428080020007008F100F0010830F2
:10018000FC007108F40C0318C928FC0BC228F1010B
:1001900000340310CE28F40C0318F107F10CF00C16
:1001A000FC0BCB28080027004C08003A0319EB2869
:1001B00021008D130630FD00FD0BDC2800000D171B
:1001C0000630FD00FD0BE22800008D170630FD0013
:1001D000FD0BE82800000800FA1FF21300300800A9
:1001E000FB14FB1FFA28FF30F300F200F100F000CF
:1001F000FA0DF20CFF3008003E20270045082900C8
:10020000A300032040302900A30003202800650834
:10021000EE006408EF005D202800E901680869022B
:100220000318C5296908660784000030673D85000A
:100230000008003A031D1E29EB01272969086607FB
:1002400084000030673D850020300002EB00EA01A9
:100250006A08043C031CBC296B08F0000530F4005C
:10026000BB2028006A08F0070030F13D1630700707
:100270008400B630713D85000008EC006508023A44
:10028000013003190030F1006508043A0130031908
:100290000030F0007008F1056508063A01300319D6
:1002A0000030F0007108F00503197F29EC195A2974
:1002B000ED135B29ED17EC195F296D1360296D179C
:1002C0006C196429ED126529ED166C1969296D12F6
:1002D0006A296D16EC186E29ED116F29ED15EC18D1
:1002E00073296D1174296D156C187829ED10792911
:1002F000ED146C187D296D107E296D149F296C19E1
:100300008329ED138429ED176C1988296D13892928
:100310006D17EC188D29ED128E29ED16EC18922927
:100320006D1293296D166C189729ED119829ED150A
:100330006C189C296D119D296D15ED106D106D08BF
:100340002900A300032027004C08043A0130031DB4
:100350000030F1004C08053A0130031D0030F00078
:100360007108F0040319B92928006D082900A300B9
:1003700003202800EA0A28292900A30103202900D4
:10038000A30103202800E90A0E29650AEE0064088B
:10039000EF005D202800E9016808690203188B2A34
:1003A0006908660784000030673D85000008003A50
:1003B000031DDC29EB01E52969086607840000308C
:1003C000673D850020300002EB00EA016A08043C2A
:1003D000031C822A6B08F0000530F400BB202800C3
:1003E0006A08F0070030F13D163070078400B6301F
:1003F000713D85000008EC006508023A01300319E0
:100400000030F1006508043A013003190030F000B3
:100410007008F1056508063A013003190030F00054
:100420007108F00503193D2AEC1B182AED13192A4F
:10043000ED17EC1B1D2A6D131E2A6D176C1B222A4B
:10044000ED12232AED166C1B272A6D12282A6D1631
:10045000EC1A2C2AED112D2AED15EC1A312A6D110A
:10046000322A6D156C1A362AED10372AED146C1AE3
:100470003B2A6D103C2A6D14652A6C1B412AED1332
:10048000422AED176C1B462A6D13472A6D17EC1A8A
:100490004B2AED124C2AED16EC1A502A6D12512AF5
:1004A0006D166C1A552AED11562AED156C1A5A2A3A
:1004B0006D115B2A6D15EC195F2AED10602AED14A1
:1004C000EC19642A6D10652A6D146D082900A300CB
:1004D000032027004C08043A0130031D0030F100CE
:1004E0004C08053A0130031D0030F0007108F0049B
:1004F00003197F2A28006D082900A3000320280083
:10050000EA0AE6292900A30103202900A301032008
:100510002800E90ACC29D32008002800E50127009B
:10052000CD010130C60028006408E500E535E53559
:10053000E535E53527004F080319A12A08302800C2
:10054000E507270046080319A82A04302800E50714
:1005500027004D080319AF2A02302800E5072700BD
:100560004E080319B52A2800E50A3E202700450851
:100570002900A3000320280065082900A300032008
:10058000D3200630FC003030FD00FD0BC52AFC0BEB
:10059000C52A000004302800E5023E202700450857
:1005A0002900A3000320280065082900A3000320D8
:1005B000D3200630FC003030FD00FD0BDD2AFC0BA3
:1005C000DD2A00000800F201F101F001F801F30159
:1005D000003008007B15FB1FF42A0130F300F20104
:1005E000F101F001FA0DF20CFF3008002800E801DB
:1005F000053068020318062B68086607860000307D
:10060000673D870020308100E80AF82A68086607FD
:1006100086000030673D87008101E80368086607AF
:10062000E9000030673DEA000A30F400F501640893
:10063000F0006508F1009F207808F0007908F100CB
:100640003030F0072800690886006A0887007008C3
:1006500081000A30F400F5016408F0006508F1003B
:100660009F2070082800E4007108E5000030710642
:10067000031D3C2B00307006031D3F2B412BE8036C
:100680000E2B08001D30FD00FD0B442B0800FB095C
:10069000FA09F909F809F80A0319F90A0319FA0A13
:1006A0000319FB0A08002800E001E1015A08E200F2
:1006B0005B08E30080305B06F00080307002031DB1
:1006C000632B00305A020318712B0130E000003018
:1006D000E1005A08003CE2005B08031C013EE30114
:1006E000E3026208E4006308E5005C08E6005D08D8
:1006F000E700F6220630DE000030DF005F08003C35
:10070000031D842B5E08003C03189F2B5E085C07CA
:1007100086005F085D3D870001305E02F00000301A
:100720005F3BF10070085C07840071085D3D850047
:10073000000881000130DE020030DF3B7E2B5C08C8
:1007400086005D088700203081006008610403197D
:10075000C52BDE01DF015E085C0784005F085D3D9C
:1007600085000008203A031DB92BDE0A0319DF0AB1
:10077000AB2B0130DE020030DF3B5E085C078600F9
:100780005F085D3D87002D30810008002000223089
:10079000FC00F801F901FA01FB01FC030319FB2B32
:1007A0000310FB0CFA0CF90CF80CF30CF20CF10C26
:1007B000F00C031CCD2BFC030319ED2B7408F80778
:1007C00075080318750FF90776080318760FFA07EE
:1007D00077080318770FFB07D12B7408F807750803
:1007E0000318750FF90776080318760FFA077708CC
:1007F0000318770FFB0708007408F8027508031C3C
:10080000750FF9027608031C760FFA027708031CAD
:10081000770FFB02F30D0730FC00730DF80DF90D97
:10082000FA0DFB0D7408731C232CF8027508031CC9
:10083000750FF9027608031C760FFA027708031C7D
:10084000770FFB02302CF80775080318750FF907AE
:1008500076080318760FFA0777080318770FFB0757
:10086000F30DFC0B0D2C720DF80DF90DFA0DFB0DAF
:100870007408731C492CF8027508031C750FF902E3
:100880007608031C760FFA027708031C770FFB0229
:10089000562CF80775080318750FF9077608031822
:1008A000760FFA0777080318770FFB07F20D07306A
:1008B000FC00720DF80DF90DFA0DFB0D7408721C99
:1008C0006F2CF8027508031C750FF9027608031CDB
:1008D000760FFA027708031C770FFB027C2CF807CF
:1008E00075080318750FF90776080318760FFA07CD
:1008F00077080318770FFB07F20DFC0B592C710DCD
:10090000F80DF90DFA0DFB0D7408721C952CF80208
:100910007508031C750FF9027608031C760FFA029E
:100920007708031C770FFB02A22CF8077508031841
:10093000750FF90776080318760FFA07770803187A
:10094000770FFB07F10D0730FC00710DF80DF90D65
:10095000FA0DFB0D7408711CBB2CF8027508031C02
:10096000750FF9027608031C760FFA027708031C4C
:10097000770FFB02C82CF80775080318750FF907E5
:1009800076080318760FFA0777080318770FFB0726
:10099000F10DFC0BA52C700DF80DF90DFA0DFB0DEA
:1009A0007408711CE12CF8027508031C750FF9021C
:1009B0007608031C760FFA027708031C770FFB02F8
:1009C000EE2CF80775080318750FF9077608031859
:1009D000760FFA0777080318770FFB07F00D07303B
:1009E000FC00700DF80DF90DFA0DFB0D7408701C6C
:1009F000072DF8027508031C750FF9027608031C11
:100A0000760FFA027708031C770FFB02142DF80704
:100A100075080318750FF90776080318760FFA079B
:100A200077080318770FFB07F00DFC0BF12C7018FB
:100A3000272D7408F80775080318750FF90776084D
:100A40000318760FFA0777080318770FFB070800DB
:100A500027004C08043A0130031D0030F1004C0817
:100A6000053A0130031D0030F0007108F00403194D
:100A7000462D28005B08E4005A08E5005C08E60003
:100A80005D08E7005E08E800FC20A02D27004C0868
:100A9000023A0130031D0030F1004C08033A0130E6
:100AA000031D0030F0007108F00403196C2D0730AD
:100AB000F00028005B08F400BB2004307007280019
:100AC000E4005A08E500E5355C08E6005D08E7004B
:100AD0005E08E800FC20A02D2700CE0128005A085F
:100AE000F000F035F0357008083EE4008D22280053
:100AF0005B08E4008D2201302700CE002800DF01D2
:100B00005E085F020318A02D5F085C0784000030B8
:100B10005D3D85000008F1007108E400E436E4362C
:100B2000E436E4368D2228005F085C07840000303C
:100B30005D3D85000008E4008D222800DF0A802D3D
:100B40000800833021009D0528005A08F000F03588
:100B5000F035700821009D0442239D149D1CB12D89
:100B6000AE2D1C08F100F0011B08F0040030F10468
:100B700008000330FC009530FD00FD0BBD2DFC0B83
:100B8000BD2D0800FB15FF3008007C18FB2DFC185C
:100B9000CC2D7C191A2EC52DA1017208031DEC2D38
:100BA0007108F2007008F1007808F000F801A11552
:100BB0007208031DEC2D7108F2007008F100F001BD
:100BC000A11121167208031DEC2D7108F200F1012C
:100BD000A115720803190E2E2108F302031D031C30
:100BE000122E0310F21BFB2DF80DF00DF10DF20D7E
:100BF000F30BF22D122E7B1B701C162EF81F162ED7
:100C0000F00A0319F10A0319F20A031D162EF20C59
:100C1000F10CF00CF30A03191A2E162E0130FC0009
:100C2000E3221D2E0230FC00EA221D2E0430FC00BF
:100C3000EC201D2E0830FC00F02000000800A1016F
:100C40007208031D342E7108F2007008F100F001E3
:100C5000A1157208031D342E7108F200F101A111D3
:100C6000211672080319422E2108F302031D031CEA
:100C7000462E0310F21B4A2EF00DF10DF20DF30B70
:100C80003A2E462E0130FC00E3224D2E0230FC00AD
:100C9000EA224D2E0430FC00EC2008007B14FB1FE0
:100CA000592EF201FA1FFF30F200F100F000FA0DA8
:100CB000F20CFF300800200072087606A100F8014F
:100CC000F90173087702031C7D2E7708FD00730875
:100CD000F7007D08F3007608FD007208F6007D0835
:100CE000F2007508FD007108F5007D08F100740838
:100CF000FD007008F4007D08F00077080319F62E57
:100D00007208FA00F217F61777087302F700031952
:100D1000B02E08307702031CA62EF7007408F900E5
:100D20007508F4007608F500F60108307702031C18
:100D3000A62EF7007408F9007508F400F5010830D4
:100D40007702031CA62E7A08F200F62E7708031904
:100D5000B02E0310F60CF50CF40CF90CF70BA92EC1
:100D6000A11FBD2EF909F409F509F609F90A0319BD
:100D7000F40A0319F50A0319F60A7908F807740842
:100D80000318740FF00775080318750FF10776083C
:100D90000318760FF207A11BD62E031CE62EF20CC9
:100DA000F10CF00CF80CF30FE62EF22E0318EA2EDD
:100DB000F809F009F109F209F80A0319F00A031910
:100DC000F10A0319F20A8030FA06EE2E0130FC0017
:100DD000C525F82E0230FC00C525F82E0430FC0095
:100DE0001F26F82E0830FC00F020F82E0030FC0002
:100DF000000008002800D9015508F1000130F0007A
:100E000071080319062FF035FF3E012F7008D80036
:100E1000530884005408850070080005F10071082B
:100E20000130031D0030F0005708F0060319322F7F
:100E30005608003C0318202FB925B925D603182FD2
:100E4000530884005408850058080005F100710813
:100E50000130031D0030F0005708F0060319322F4F
:100E6000FF30D9005908F0000800710DF80DF90D98
:100E70007408F8027508031C750FF902F00DF10DE6
:100E80000F30FC00710DF80DF90D7408701C4E2F19
:100E9000F8027508031C750FF902532FF80775083F
:100EA0000318750FF907F00DF10DFC0B422F7018A8
:100EB0005F2F7408F80775080318750FF90700000D
:100EC00008002000FB017308031D77080319B72FE2
:100ED00072087606FA007708F3077E30031C742F39
:100EE000F3020318BA2F772FF302031CBD2F7208E9
:100EF000F8007108FC007008FD00F817F6170310E1
:100F0000F201F101F0011830A1007D1C912F74084D
:100F1000F00775080318750FF10776080318760FA8
:100F2000F207F20CF10CF00CF80CFC0CFD0C0310A9
:100F3000A10B852FF21BA12FF80DF00DF10DF20D75
:100F4000F3037B1B701CB32FF81FB32FF00A031998
:100F5000F10A0319F20A031DB32FF20CF10CF00C85
:100F6000F30A0319BA2FFA1FF2130030BF2F013012
:100F7000E322BF2F0230F020BF2F0430EA2200000E
:100F8000080020007008F8007108F0007208F100F5
:100F90007308F200F301FB01FC019E30F300FA013B
:100FA000F21FDE2FF809F009F109F209F80A031916
:100FB000F00A0319F10A0319F20AFA170230FC00C9
:100FC000C525080020007008F800FB01FC019E30D8
:100FD000F300FA01F201F101F0010230FC00C52535
:100FE0000800A1302700C8000530C9005A30CA00E7
:100FF0000430CB00F03021009E009D011D1408003C
:1010000064002700A001A1012500501C0F28260024
:101010006D082700A00726006E082700A13D2500C7
:10102000D01C172827002A08A0072B08A13D25005F
:10103000501D1F2827002808A0072908A13D2500CA
:10104000D01D272827002608A0072708A13D250036
:10105000501E2F2827002C08A0072D08A13D250091
:10106000D01E372827003008A0073108A13D2500F1
:10107000501F3F2827002E08A0072F08A13D27005A
:101080008030273AF000803021067002031D4A2884
:1010900020080F3C03186C2832302007F000003085
:1010A000213DF1007008A0007108A100700828001F
:1010B000DA007108DB00BD30DC000330DD00803178
:1010C0005323883127003E08B6003F08B7002E3072
:1010D000B8004008B900982820082800DA00270046
:1010E00021082800DB00BD30DC000330DD0080314A
:1010F0005323883127003F08203A031982283F08EC
:10110000B60084283030B6002E30B7004008203AB0
:1011100003198D284008B8008F283030B8004108E6
:10112000203A031996284108B90098283030B900B0
:101130006608043A0130031D0030F1006608053AE4
:101140000130031D0030F0007108F0040319DE289F
:1011500025005108013A031DB12804302800D300AE
:10116000B42828000630D3005308DA001030DB0022
:10117000A830DC000030DD000230DE0080312825A0
:10118000883128005308DA005830DB00A030DC003A
:101190000030DD000230DE00803128258831280053
:1011A0005308DA002830DB00B630DC000330DD0005
:1011B0000430DE008031282588315D29270066084B
:1011C000023A0130031D0030F1006608033A013095
:1011D000031D0030F0007108F004031924292500D4
:1011E0005108013A031DF7282800D301FA282800E6
:1011F0000130D3005308DA000930DB006D30DC0029
:101200000030DD000230DE008031282588312800E2
:101210005308DA000F30DB006A30DC000030DD00FC
:101220000230DE0080312825883128005308DA009A
:101230000B30DB00B630DC000330DD000430DE00B4
:101240008031282588315D2927006608013A031D71
:101250005D2925005108013A031D31292800D301D9
:10126000342928000130D3005308DA000930DB00AC
:10127000A330DC000030DD000230DE0080312825A4
:10128000883128005308DA000F30DB00A630DC007C
:101290000030DD000130DE00803128258831280053
:1012A0005308DA000B30DB00B630DC000330DD0021
:1012B0000430DE0080312825883164002700A00139
:1012C000A10125004F1C692927002408A007250833
:1012D000A13D2500CF1C712927002208A007230863
:1012E000A13D25004F1D792927005408A007550866
:1012F000A13D2500CF1D812927005208A0075308D2
:10130000A13D25004F1E892927005008A00751083C
:10131000A13D2500CF1E912927005608A007570898
:10132000A13D25004F1F992927005808A0075908FB
:10133000A13D270020082800DA0027002108280006
:10134000DB00BD30DC000330DD0080315323883109
:1013500027003F08B6004008B7004108B80042081F
:10136000B9006608043A0130031D0030F100660838
:10137000053A0130031D0030F0007108F004031934
:10138000F72925005108013A031DCA290630280013
:10139000D300CD2928000430D3005308DA001030E0
:1013A000DB006C30DC000230DD000230DE0080311A
:1013B0002825883128005308DA005830DB006930CE
:1013C000DC000230DD000230DE008031282588316B
:1013D00028005308DA002830DB00B630DC00033088
:1013E000DD000430DE00803128258831762A270090
:1013F0006608023A0130031D0030F1006608033A26
:101400000130031D0030F0007108F00403193D2A7B
:1014100025005108013A031D112A01302800D3008C
:10142000132A2800D3015308DA000930DB006130A9
:10143000DC000230DD000230DE00803128258831FA
:1014400028005308DA000F30DB005E30DC00023089
:10145000DD000230DE008031282588312800530865
:10146000DA000B30DB00B630DC000330DD00043086
:10147000DE00803128258831762A27006608013A67
:10148000031D762A25005108013A031D4B2A01301D
:101490002800D3004D2A2800D3015308DA00093070
:1014A000DB005B30DC000230DD000230DE0080312A
:1014B0002825883128005308DA000F30DB0064301B
:1014C000DC000230DD000130DE008031282588316B
:1014D00028005308DA000B30DB00B630DC000330A4
:1014E000DD000430DE0080312825883164000800EA
:1014F0002000FB01FA01F9018030F800F10CF00C3A
:10150000031C8B2A7408F90775080318750FFA076E
:101510000318FB0A0310F01F932A7408FA077508D2
:101520000318750FFB07FB0CFA0CF90CF80C031CE5
:101530007E2A7B08F3007A08F2007908F100780827
:10154000F00008002000FB0173080319DE2A72086E
:10155000FA00F2178E30F302F31FE12AF309F30ABF
:1015600008307302031CC42AF300F10D7208F10065
:10157000F20108307302031CC42AF300F10DF101DB
:101580007308031D0310CC2A73080319CC2A031017
:10159000F20CF10CF30BC72A7B1B711CD62A031C1F
:1015A000D62AF10A0319F20AF21BED2AFA1FF02AD1
:1015B000F209F109F10A0319F20AF02AF201F10124
:1015C000F02A7B14FB1FF32AF201FA1FF32AFF30E3
:1015D000F200F100FA0DF20CF32A0130FC00F52ABA
:1015E0000030FC00F52AFF30FC00FC080319FB2A40
:1015F00080314E2688317108F0007208F100080031
:101600007408003A031D192B7508003A031D192BA5
:101610007608003A031D192B7708003A031D192B91
:10162000FF30F000FF30F1007F30F200FF30F300B8
:10163000BB2B200077080319A72B73080319AC2BC9
:10164000720876068039FA00F217F617A1017208BF
:10165000F8007108FC007008FD007408FD027508B0
:10166000031C750FFC027608031C760FF802F801C4
:10167000FC01FD01031C432B0310F20CF10CF00CD8
:10168000F80C0130A1007708F302031C4D2B7E30CB
:101690002107F3070318B12B522B7E302107F307E4
:1016A000031CB62B1830FA07FD0DFC0DF80DF00DDC
:1016B000F10DF20DA10D7408F0027508031C750FF1
:1016C000F1027608031C760FF202760DA104211CAC
:1016D0006B2B7D14762B7408F00775080318750FB3
:1016E000F10776080318760AF2077D10FA031F3017
:1016F0007A05031D542B7B1B7D1C9D2B0310F00DC5
:10170000F10DF20DA10D7408F0027508031C750FA0
:10171000F1027608031C760FF202760D21040139DE
:10172000FD070318FC0A0319F80A031D9D2BF80C8A
:10173000FC0CFD0CF30A0319B12BFA1FF8137808FF
:10174000F2007C08F1007D08F0000030BA2B013077
:101750008031C2258831BA2B02308031E3228831B2
:10176000BA2B04308031F0208831BA2B0830803118
:10177000EA22883100000800813022009700171B00
:10178000C22BBF2B2800DA018031A12588317008D7
:101790002800D3007108D4008030033AF200803072
:1017A00071067202031DD62B7008E83C031CDD2B6A
:1017B0005308F0005408F1001C2C823022009700DE
:1017C000171BE32BE02B2800DA018031A12588319B
:1017D00070082800D3007108D4008030033AF2006A
:1017E000803071067202031DF72B7008E83C031C61
:1017F000002C5308F0005408F100F035F10D1C2CBA
:10180000833022009700171B062C032C2800DA01D6
:101810008031A125883170082800D3007108D400D8
:101820007008F2007108F300F235F30DF235F30D94
:101830007208F0007308F100080081302200970060
:10184000171B232C202C01302800DA008031A12521
:10185000883170082800D3007108D4008030033A22
:10186000F200803071067202031D382C7008E83CCB
:10187000031C422C2600C50128005308F000540820
:10188000F100952C823022009700171B482C452C24
:1018900001302800DA008031A12588317008280045
:1018A000D3007108D4008030033AF2008030710612
:1018B0007202031D5D2C7008E83C031C692C260095
:1018C000C50128005308F0005408F100F035F10D6F
:1018D000952C833022009700171B6F2C6C2C013045
:1018E0002800DA008031A125883170082800D30053
:1018F0007108D4008030033AF20080307106720221
:10190000031D842C7008E83C03188A2C0130260043
:10191000C5008C2C2600C50128005308F00054088F
:10192000F100F035F10DF035F10D08007408003AC2
:10193000031DAF2C7508003A031DAF2C7608003A42
:10194000031DAF2C7708003A031DAF2CFF30F000C9
:10195000FF30F100FF30F2007F30F3004B2D20000C
:10196000FC01F71BFC0AFD01FB01FA01F901F8017A
:1019700073087204710470040319442D7308770608
:10198000A000A01BFD09F71FD02CF409F509F609EA
:10199000F709F40A0319F50A0319F60A0319F70AF5
:1019A000F31FDD2CF009F109F209F309F00A03191C
:1019B000F10A0319F20A0319F30A73087704A00065
:1019C000A01B002D8031FC238831FC1B1D2DFD1F29
:1019D000442DF009F109F209F309F00A0319F10A9B
:1019E0000319F20A0319F30AF809F909FA09FB09BC
:1019F000F80A0319F90A0319FA0A0319FB0A442D14
:101A0000F71F172DF31B112D7308FB007208FA0046
:101A10007108F9007008F800F301F201F101F0011A
:101A2000E72CF301F201F101F001F00A0034F309AF
:101A3000F209F109F009FC17E22CF80A0319F90A76
:101A40000319FA0A0319FB0A74087802031DE72C2C
:101A500075087902031DE72C76087A02031DE72C2E
:101A600077087B02031DE72CFB01FA01F901F8015D
:101A7000F00A0319F10A0319F20A0319F30AF31F12
:101A8000E72CA0012016FF34A0017C1C4A2D8031D8
:101A900047238831003E080020007008F8007108D4
:101AA000F000F101F201F301FB01FC019630F300BB
:101AB000FA01F01F612DF809F009F80A0319F00A7C
:101AC000FA177008F1007808F000F801F20180318F
:101AD0001F2688310800A0302800D5000F30D6001E
:101AE000D701D801A030F0000F30F1000030F20033
:101AF0000030F3005308F4005408F500F601F70134
:101B00008031C623883170082800D5007108D600BE
:101B10007208D7007308D80000307302031D9A2D95
:101B200000307202031D9A2D02307102031D9A2D9E
:101B3000B230700203189D2DCC2DB230D502023088
:101B4000D63B0030D73BD83B0530F0007008031976
:101B5000AF2DD836D70CD60CD50CFF3EA72D550887
:101B6000F0005608F1005708F2005808F300013061
:101B7000D5020030D63BD73BD83B700871047204C5
:101B800073040319CC2D00000000000000000000C9
:101B9000000000000000AF2D080080313E20883199
:101BA000270045082900A3008031032088318030B8
:101BB0002900A30080310320883128005308290020
:101BC000A3008031032088318031D3208831080080
:101BD0008030F0008030280054067002031DF22D82
:101BE0005308503C031CF72DF001F101CA2E803040
:101BF000F000803054067002031D002E5308AB3CE9
:101C0000031C072EF430D3070030D43DC62E80309D
:101C1000013AF000803054067002031D112E530863
:101C2000483C031C182EFE30D3070030D43DC62E8E
:101C30008030023AF000803054067002031D222EDC
:101C40005308463C031C292E1830D3070130D43DDD
:101C5000C62E8030033AF000803054067002031D17
:101C6000332E5308343C031C3A2E2930D30701305D
:101C7000D43DC62E8030043AF00080305406700205
:101C8000031D442E53084C3C031C4B2E3630D30707
:101C90000130D43DC62E8030083AF0008030540622
:101CA0007002031D552E5308853C031C5C2EAE307C
:101CB000D3070130D43DC62E80300C3AF00080307E
:101CC00054067002031D662E5308FA3C031C6D2E49
:101CD000E430D3070130D43DC62E8030123AF000F4
:101CE000803054067002031D772E53080F3C031CEE
:101CF0007E2E1230D3070230D43DC62E8030163AE5
:101D0000F000803054067002031D882E5308E63C14
:101D1000031C8F2E8830D3070230D43DC62E80306E
:101D20001B3AF000803054067002031D992E5308B0
:101D3000EA3C031CA02EE730D3070230D43DC62E68
:101D40008030213AF000803054067002031DAA2E24
:101D50005308363C031CB12E2030D3070330D43D4A
:101D6000C62E8030293AF000803054067002031DE0
:101D7000BB2E5308043C031CC22E4830D30703304B
:101D8000D43DC62E5C30D3070330D43D5308F00059
:101D90005408F10008002000FA017308031D7A14AA
:101DA0007708031DFA147A080319162F033A03194A
:101DB000E12E7A18DE2EF61F142F122FF21F122F8B
:101DC000142F72088039FA00F21376088039F6135E
:101DD0007A060319EF2E7A080319122F142F7708A9
:101DE00073020319F62E031C0A2F0E2F76087202B7
:101DF0000319FD2E031C0A2F0E2F750871020319FB
:101E0000042F031C0A2F0E2F740870020319162FBB
:101E100003180E2FFA080319142F122FFA080319AA
:101E2000122F142F031408000310080003140315C5
:101E30000800080028003718202F22000E10222F3B
:101E400022000E14270064082800D300270065082C
:101E50002800D4006B25080025005808003A031D0F
:101E60006A2F28003718372F22008D11392F2200B2
:101E70008D152800B7183F2F22000C11412F22008A
:101E80000C1528003719472F22000D12492F220068
:101E90000D162800B7194F2F22008C11512F220048
:101EA0008C152800371A572F22008D12592F220027
:101EB0008D162800B71A5F2F22008C12612F220086
:101EC0008C162800371B672F22000C12692F220066
:101ED0000C16A22F28003718702F22008D15722F94
:101EE00022008D112800B718782F22000C157A2FA8
:101EF00022000C1128003719802F22000D16822F86
:101F000022000D122800B719882F22008C158A2F65
:101F100022008C112800371A902F22008D16922F44
:101F200022008D122800B71A982F22008C169A2FA3
:101F300022008C122800371BA02F22000C16A22F83
:101F400022000C12270064082800D300270065082F
:101F50002800D4006B25080027004C08013C03181A
:101F6000B62FAF302800D300CD25C82F27004C084E
:101F7000013A031DC82F0130CF00CE012800E40133
:101F800080318D2288312800E40180318D22883112
:101F900008000D302800D3000030D400D5011930DE
:101FA000D600D7018031FA2688317008B7000D308D
:101FB000D3000030D4000130D5001930D600D7014D
:101FC0008031FA2688317008B7040D30D300003014
:101FD000D4000230D5001930D600D7018031FA265E
:101FE00088313708F0040319F82F01302600E1008A
:101FF0000800543455344E34453400346C340034C5
:102000007408003A031D0D287508003A031D0D28B9
:10201000FF30F0007F30F10067282000FD01F9015A
:10202000F801710870040319003471087506FA008C
:10203000FA1BFD09FB01F51F2228F409F509F40A32
:102040000319F50AF11F2928F009F109F00A03190B
:10205000F10A71087504FA00FA1B3E288031352711
:1020600090317B185328FD1F0034F009F109F00A64
:102070000319F10AF809F909F80A0319F90A0034F1
:10208000F51F4F28F11B4B287108F9007008F80064
:10209000F101F0013328F101F001F00A0034F109F7
:1020A000F009FB0A3028F80A0319F90A74087802C3
:1020B000031D332875087902031D3328F901F8013F
:1020C000F00A0319F10AF11F33280000FF34080059
:1020D000280037186E2822008E13702822008E17D1
:1020E0002800B718762822008E11782822008E1535
:1020F000280037197E2822000E13802822000E1790
:102100002800B719862822000E11882822000E15F3
:102110002800371A8E2822008E12902822008E1650
:102120002800B71A962822008E10982822008E14B4
:102130002800371B9E2822000E12A02822000E160F
:10214000270064082800D300270065082800D40071
:1021500088316B259031080000302800BF00003026
:10216000C0004830C1008530C200640021006B0807
:10217000003A0130031D0030F1004F08013A0130F0
:10218000031D0030F0007008F1058030280038068B
:10219000F00080307002031DCF280A303702013072
:1021A000031C0030F0007108F00503199529250083
:1021B0004E08003A031D912927006608043A0130B1
:1021C000031D0030F1006608053A0130031D0030A0
:1021D000F0007108F00403191E2926003608013AA0
:1021E000031D012904302800DA001030DB00A03084
:1021F000DC000130DD000830DE0080312825903120
:102200000F2904302800DA001030DB00BB30DC007E
:102210000130DD000830DE008031282590310630A5
:102220002800DA001030DB00B230DC000130DD00C5
:102230000830DE008031282590319129270066087A
:10224000023A0130031D0030F1006608033A013004
:10225000031D0030F0007108F00403195E29260008
:102260003608013A031D42292800DA010930DB0053
:10227000A930DC000130DD000830DE008031282587
:1022800090314F292800DA010930DB005530DC009D
:102290000130DD000830DE0080312825903101302A
:1022A0002800DA000930DB004C30DC000130DD00B2
:1022B0000830DE00803128259031912927006608FA
:1022C000013A031D912926003608013A031D76299B
:1022D0002800DA010930DB004430DC000130DD0089
:1022E0000730DE0080312825903183292800DA016B
:1022F0000930DB005E30DC000130DD000730DE003D
:1023000080312825903101302800DA000930DB00C7
:102310006630DC000130DD000730DE00803128252A
:10232000903101302500CE009F2925004E08013A4A
:10233000031D9D298831002090312500CE016400C5
:102340002800380825005506031DA929540828002F
:10235000370603198C2D280037082500D4002800E3
:1023600038082500D50026003608003A031D072A44
:10237000803028003806F00080307002031DC2292A
:1023800064303702031CE32905303707F0000030C2
:10239000383DF1007008B7007108B8007008DA0025
:1023A0007108DB00BD30DC000330DD0080315323D9
:1023B000903127003F08B6004008B7004108B80038
:1023C0005730B900062A28003708DA003808DB0041
:1023D000BD30DC000330DD00803153239031270015
:1023E0004108203A0319F7294108B600F92930308D
:1023F000B6002E30B7004208203A0319022A4208DC
:10240000B800042A3030B8005730B9003E2A803076
:1024100028003806F0008030033A7002031D122AAB
:10242000E73037020318292A3708DA003808DB00BA
:10243000BD30DC000330DD008031532390312700B4
:102440004008B6004108B7004208B8005730B9004C
:102450003E2A28003708DA003808DB00BD30DC00EF
:102460000330DD0080315323903127003F08B60050
:102470004008B7004108B8004208B9006608043AAD
:102480000130031D0030F1006608053A0130031DDC
:102490000030F0007108F00403195C2A2800DA010A
:1024A0004030DB00B630DC000330DD000430DE00FD
:1024B0008031282590316E2A27006608003A0319DA
:1024C0006E2A2800DA010430DB00B630DC0003306D
:1024D000DD000430DE0080312825903164002500C5
:1024E0004E08013A031D8C2D5008003A0130031D9F
:1024F0000030F1004F08003A0130031D0030F000B9
:102500007108F00503198C2A280039082700B40047
:1025100028003A082700B50027003408F0003508E5
:10252000F10088314C25903170082800CB007108EB
:10253000CC007208CD007308CE000030F4000030EB
:10254000F5004830F6008530F7004B08F0004C08E5
:10255000F1004D08F2004E08F3008831002390315D
:1025600070082800C7007108C8007208C900730805
:10257000CA004B08F4004C08F5004D08F6004E0860
:10258000F7000030F0000030F1004830F2008530F4
:10259000F30088310023903128004708F4004808F0
:1025A000F5004908F6004A08F70080315B269031B3
:1025B00070082800C7007108C8007208C9007308B5
:1025C000CA0026006F08F0008031E2279031280011
:1025D0004708F4004808F5004908F6004A08F700E3
:1025E0008031612790310030F4000030F500203058
:1025F000F6008230F7008831002390311F30F4005C
:102600008530F5006B30F6007B30F70080316127B4
:1026100090310030F4000030F5000030F6007F30DB
:10262000F70080315B2690317008F4007108F500E6
:102630007208F6007308F7000030F0000030F10077
:102640000030F2007F30F3008831002390317008B1
:102650002800CF007108D0007208D1007308D200A2
:102660004F08BF005008C0005108C1005208C20006
:102670003908F0003A08F10088314C259031700893
:102680002800CB007108CC007208CD007308CE0082
:102690000030F4000030F5004830F6008530F700D7
:1026A0004B08F0004C08F1004D08F2004E08F30012
:1026B0008831002390310030F4000030F500003004
:1026C000F6008030F70080315B26903170082800DA
:1026D000C7007108C8007208C9007308CA004B0817
:1026E000F4004C08F5004D08F6004E08F7000030E5
:1026F000F0000030F1004830F2008530F3008831FE
:102700000023903128004708F4004808F5004908E4
:10271000F6004A08F70080315B2690317008F4001B
:102720007108F5007208F6007308F7000030F00039
:102730000030F1000030F2008130F30088310023D6
:10274000903170082800C3007108C4007208C500E9
:102750007308C6000030F4000030F5000030F600C9
:102760007F30F7004F08F0005008F1005108F200E8
:102770005208F3008831CB2690310130031C003021
:10278000F00070080319CD2B00302800BF00003086
:10279000C0000030C1007F30C20028000030F400CB
:1027A0000030F5000030F6007F30F7004308F000FD
:1027B0004408F1004508F2004608F3008831CB26B2
:1027C00090310130031C0030F00070080319F12B28
:1027D00000302800C3000030C4000030C5007F3046
:1027E000C60028003708F0003808F10088314C2571
:1027F000903128003F08F4004008F5004108F60039
:102800004208F70080316127903128004308F40026
:102810004408F5004508F6004608F70080316127B6
:1028200090318831A222903170082800BB007108D5
:10283000BC003F08F0004008F1004108F2004208E7
:10284000F3004308F4004408F5004508F600460884
:10285000F7008031612790310030F4000030F5003E
:102860004830F6008530F70080316127903188319B
:10287000A222903170082800BD007108BE0080308F
:102880007106F20080307202031D482C6430700221
:10289000031C4E2C6330BD000030BE0026003608FD
:1028A000003A031DA22C803028003C06F000803046
:1028B0007002031D5D2C64303B02031C7E2C05302E
:1028C0003B07F00000303C3DF1007008BB00710890
:1028D000BC007008DA007108DB00BD30DC0003309A
:1028E000DD0080315323903127003F08B6004008B7
:1028F000B7004108B8005730B900A12C28003B08A8
:10290000DA003C08DB00BD30DC000330DD00803144
:102910005323903127004108203A0319922C410893
:10292000B600942C3030B6002E30B7004208203A62
:1029300003199D2C4208B8009F2C3030B800573046
:10294000B900D92C803028003C06F0008030033AD2
:102950007002031DAD2CE7303B020318C42C3B086A
:10296000DA003C08DB00BD30DC000330DD008031E4
:102970005323903127004008B6004108B7004208B1
:10298000B8005730B900D92C28003B08DA003C08C1
:10299000DB00BD30DC000330DD008031532390319B
:1029A00027003F08B6004008B7004108B8004208B9
:1029B000B9006608043A0130031D0030F1006608D2
:1029C000053A0130031D0030F0007108F0040319CE
:1029D000F82C04302800DA004030DB00B630DC0090
:1029E0000330DD000430DE00803128259031292DB0
:1029F00027006608023A0130031D0030F100660826
:102A0000033A0130031D0030F0007108F00403198F
:102A1000172D2800DA010D30DB00B630DC00033062
:102A2000DD000430DE00803128259031292D27007B
:102A30006608003A0319292D2800DA010C30DB0062
:102A4000B630DC000330DD000430DE0080312825A4
:102A5000903128003D08DA003E08DB00BD30DC0084
:102A60000330DD0080315323903127004108B60048
:102A70004208B7006608043A0130031D0030F10037
:102A80006608053A0130031D0030F0007108F004BB
:102A90000319592D06302800DA004C30DB00B6301F
:102AA000DC000330DD000230DE008031282590316B
:102AB0008C2D27006608023A0130031D0030F1001A
:102AC0006608033A0130031D0030F0007108F0047D
:102AD0000319792D01302800DA000E30DB00B63002
:102AE000DC000330DD000230DE008031282590312B
:102AF0008C2D27006608013A031D8C2D013028001B
:102B0000DA000D30DB00B630DC000330DD000230CF
:102B1000DE00803128259031640008006400280020
:102B2000380825005706031D982D5608280037063B
:102B300003195B2E280037082500D6002800380826
:102B40002500D700003028003806031DA92D0030CD
:102B50003706031DEB2D27006608043A0130031DDC
:102B60000030F1006608053A0130031D0030F00026
:102B70007108F0040319CB2D02302800DA00403030
:102B8000DB004530DC000030DD000430DE00803149
:102B900028259031E72D27006608003A0319DF2D1C
:102BA00001302800DA000430DB004030DC00003067
:102BB000DD000430DE00803128259031E72D27002C
:102BC0006608003A031DE72D22000D178D1725001A
:102BD000D601D7015B2E28003708DA003808DB0061
:102BE000BD30DC000330DD008031532390312700FD
:102BF0004008B6002E30B7004108B8004208B900BE
:102C00006608043A0130031D0030F1006608053AF9
:102C10000130031D0030F0007108F00403191F2E6D
:102C200002302800DA004030DB00B630DC00033030
:102C3000DD000430DE008031282590315B2E270036
:102C40006608003A0319332E01302800DA000430F8
:102C5000DB00B630DC000330DD000430DE00803104
:102C6000282590315B2E27006608003A031D5B2E55
:102C70008030F0008030280038067002031D422E9C
:102C80003708963C031C482E22000D138D175B2E2F
:102C90008030F0008030280038067002031D522E6C
:102CA0003708FA3C031C582E20000D138D135B2EA1
:102CB00020000D178D1364000800640088311D2466
:102CC00090317008B7007108B8000030B81BFF30B1
:102CD000B900BA008831BC2390317008BB0071087C
:102CE000BC000030BC1BFF30BD00BE002600350814
:102CF000013A031D9C2E28003708F0003808F10027
:102D00000330F4000030F5008831782290317008EB
:102D10002800D3007108D4008831E825903188312B
:102D20004C25903170082800BF007108C00072085F
:102D3000C1007308C200B92E28003708F000380817
:102D4000F1003908F2003A08F3000330F400F5010D
:102D5000F601F7018031C62390318031C1279031CF
:102D600070082800BF007108C0007208C100730815
:102D7000C20080303E06F00080303A067002031D2B
:102D8000CB2E39083D02031DCB2E38083C02031D13
:102D9000CB2E37083B02031CD42EE730B70003309C
:102DA000B800B901BA011E2F3B083707F0003C08F4
:102DB000383DF1003D08393DF2003E083A3DF30050
:102DC0006430F400F501F601F7018031C62390313B
:102DD00028003708F4003808F5003908F6003A08EA
:102DE000F7003B08F4023C08F53B3D08F63B3E0883
:102DF000F73B88319624903170082800B70071089D
:102E0000B8007208B9007308BA008030F40080304E
:102E100073067402031D162F7208003C031D162F43
:102E20007108033C031D162F7008E73C03181E2F82
:102E3000E730B7000330B800B901BA0126003708FF
:102E4000F0008031E227903128003F08F40040086C
:102E5000F5004108F6004208F70080316127903103
:102E60000030F4000030F5007A30F6008830F700CA
:102E700088310023903170082800BF007108C0001D
:102E80007208C1007308C200F430F400FD30F50090
:102E90003430F6007F30F70088310023903170081D
:102EA0002800BF007108C0007208C1007308C2008A
:102EB00026003608013A031D862F28003F08F0003F
:102EC0004008F1004108F2004208F3003F08F40016
:102ED0004008F5004108F6004208F70080316127FC
:102EE00090310030F4000030F5004830F6008430B6
:102EF000F70088310023903170082800BF00710866
:102F0000C0007208C1007308C200AE2F28003F083D
:102F1000F0004008F1004108F2004208F3003F08C9
:102F2000F4004008F5004108F6004208F70080313F
:102F3000612790310030F4000030F5002030F600B9
:102F40008130F70088310023903170082800BF00DD
:102F50007108C0007208C1007308C2003F08F00089
:102F60004008F1004108F2004208F3000030F4008C
:102F70000030F5000030F6007E30F70080315B262F
:102F8000903170082800BF007108C0007208C100AD
:102F90007308C2008831A222903170082700E00037
:102FA0007108E100803028003A06F000803070029D
:102FB000031DE42F00303902031DE42F00303802D6
:102FC000031DE42F643037020318EC2FE73027008D
:102FD000E2000330E300F42F280037082700E20066
:102FE000280038082700E300080027006C082300A9
:102FF000910092019513151315141308F0000800A1
:103000002800B501B6016430270067022800B0002F
:1030100000302700683B2800B1002700E001E101F3
:10302000640025006B08003A0130031D0030F100F8
:103030006C08013A0130031D0030F0007108F00502
:103040000319662890315D26983180306106F000C2
:1030500080307002031D2E280A306002031C652890
:10306000250050082800B70088312C27983125000A
:103070004F082800B700903168209831250051088A
:103080002800B70088311A27983101302500EB005D
:103090008831AC27983125006D08F0008031E22797
:1030A000983126003808F4003908F5003A08F6008F
:1030B0003B08F7008031612798318831A22298318E
:1030C00070082500EE007108EF00042C783028000D
:1030D000B200AF0132082F020318CF2820008D184C
:1030E00073287614742876100D197828031479281B
:1030F000031076187F2803187F28F6108028F6140E
:1031000020000D188528031486280310031C8D2821
:103110002700691C8D2876148E287610F6189428BE
:1031200076189428031095280314031CA1288831CD
:10313000C927983126006108013A031DA128E10141
:10314000042C90315D269831803028003606F0003E
:103150008030270061067002031DB1286008280036
:1031600035020318C328270060082800B50027008F
:1031700061082800B600270062082800B300270075
:1031800063082800B4001030FC009430FD002800D3
:10319000FD0BC728FC0BC7280000AF0A6A28640093
:1031A00080303606F00080307002031DD92864306C
:1031B0003502031CF92805303507F0000030363D94
:1031C000F1000A30F4000030F50090310020983111
:1031D00070082800B5007108B6000A30F40000300D
:1031E000F50088317822983170082800B500710800
:1031F000B60035082600E200280036082600E30065
:10320000803028003606F00080307002031D0A2945
:103210000A30350203180E29B301B4013308B70090
:103220003408B80090318E2598318030260063062E
:10323000F10080307102031D1F290A306202013043
:10324000031C0030F10025006D08003C013003181C
:103250000030F0007108F005031947296D08F000EF
:103260008031E227983126003808F4003908F5004B
:103270003A08F6003B08F700803161279831883121
:10328000A222983170082500EE007108EF0080300E
:1032900028003406F0008030270068067002031D05
:1032A00054296708280033020130031C0030F00065
:1032B000700826006505F500803025005306F300F0
:1032C0008030280034067302031D69293308250065
:1032D00052022500013003180030F3005208280084
:1032E0003302F100250053082800343BF2008030FF
:1032F0003106F000803072067002031D81297108CA
:103300003002013003180030F00070087305F4003B
:1033100080303406F3008030250053067302031D0D
:103320009429520828003302280001300318003085
:10333000F300330825005202F1002800340825006C
:10334000533BF200803028003106F00080307206D6
:103350007002031DAD2971083002013003180030DE
:10336000F0007308F00570087404F100250053089C
:10337000033A031DBD29E73052060130031D00301A
:10338000F0007108F0047508F0050319CA2901302E
:103390002600E40020008D18CF297614D02976105D
:1033A0000D19D4290314D52903107618DB29031825
:1033B000DB29F610DC29F61420000D18E12903148E
:1033C000E2290310031CE9292700691CE929761466
:1033D000EA297610F618F0297618F0290310F12959
:1033E0000314031CFD298831C92798312600610880
:1033F000013A031DFD29E101042C26006208280082
:10340000B700260063082800B8003308B900340864
:10341000BA009031AC20983120008D18112A761412
:10342000122A76100D19162A0314172A031076187B
:103430001D2A03181D2AF6101E2AF61420000D1846
:10344000232A0314242A0310031C2B2A2700691C97
:103450002B2A76142C2A7610F618322A7618322A5D
:103460000310332A0314031C3F2A8831C9279831DB
:1034700026006108013A031D3F2AE101042C2600C1
:1034800064004508013A031D042C27006608043A2D
:103490000130031D0030F1006608053A0130031DBC
:1034A0000030F0007108F0040319282B02302800C6
:1034B000DA001030DB003C30DC000330DD00083087
:1034C000DE008031282598310330FB000830FC00F5
:1034D0007730FD00FD0B6A2AFC0B6A2AFB0B6A2A77
:1034E00002302800DA001030DB004630DC00033008
:1034F000DD000830DE008031282598310B30FB00DC
:103500002630FC005D30FD00FD0B842AFC0B842A74
:10351000FB0B842A00000000640002302800DA005F
:103520001030DB005830DC000330DD000830DE00F6
:103530008031282598310730FB001730FC006A30B5
:10354000FD00FD0BA12AFC0BA12AFB0BA12A000008
:10355000640002302800DA001030DB004F30DC005D
:103560000330DD000830DE008031282598310B3033
:10357000FB002630FC005D30FD00FD0BBD2AFC0B7E
:10358000BD2AFB0BBD2A00000000640002302800A9
:10359000DA001030DB00BD30DC000230DD00083026
:1035A000DE008031282598310730FB001730FC0001
:1035B0006A30FD00FD0BDA2AFC0BDA2AFB0BDA2A53
:1035C0000000640002302800DA001030DB00E23036
:1035D000DC000030DD000830DE0080312825983125
:1035E0000B30FB002630FC005D30FD00FD0BF62AA1
:1035F000FC0BF62AFB0BF62A0000000064000230E8
:103600002800DA001030DB00D930DC000030DD00AB
:103610000830DE008031282598310330FB00083067
:10362000FC007730FD00FD0B132BFC0B132BFB0B69
:10363000132B02302800DA001030DB00D030DC0021
:103640000030DD000830DE00803128259831F62B6F
:1036500027006608003A0319F62B01302800DA002B
:10366000DB012030DC000130DD000830DE0080317D
:10367000282598310330FB000830FC007730FD002E
:10368000FD0B402BFC0B402BFB0B402B013028008B
:10369000DA00DB013B30DC000130DD000830DE0009
:1036A0008031282598310B30FB002630FC005D303E
:1036B000FD00FD0B592BFC0B592BFB0B592B00006C
:1036C0000000640001302800DA00DB013230DC0049
:1036D0000130DD000830DE008031282598310730C8
:1036E000FB001730FC006A30FD00FD0B752BFC0B56
:1036F000752BFB0B752B0000640001302800DA00ED
:10370000DB012930DC000130DD000830DE008031D3
:10371000282598310B30FB002630FC005D30FD0081
:10372000FD0B902BFC0B902BFB0B902B0000000053
:10373000640001302800DA00DB01BD30DC0000301D
:10374000DD000830DE008031282598310730FB008D
:103750001730FC006A30FD00FD0BAC2BFC0BAC2BD2
:10376000FB0BAC2B0000640001302800DA00DB0109
:10377000B430DC000030DD000830DE008031282568
:1037800098310B30FB002630FC005D30FD00FD0B56
:10379000C72BFC0BC72BFB0BC72B000000006400E2
:1037A00001302800DA00DB01AB30DC000030DD0046
:1037B0000830DE008031282598310330FB000830C6
:1037C000FC007730FD00FD0BE32BFC0BE32BFB0B28
:1037D000E32B01302800DA00DB01C630DC000030CA
:1037E000DD000830DE00803128259831640010307B
:1037F0002500D6002730D70028003308B70034084A
:10380000B80090318E259831080028002F08230039
:10381000910092012800300823009300151395139E
:1038200015150B08F0008B1355309600AA30960042
:103830009514F01B1D2C8B131E2C8B171511951C2A
:10384000222C1F2C08002500D001CF012800B70131
:1038500088312C27983125004F082800B700903177
:1038600068209831270064082800D30027006508E5
:103870002800D40088316B259831080023240130BA
:103880002500D10001302800B70088311A2798316F
:10389000FF30AF00B0010524FE302800AF00B001BA
:1038A0000524FD302800AF000130B0000524FC30B5
:1038B0002800AF00B0010524FB302800AF00B001A4
:1038C00005248831002098312500CE0122008C1378
:1038D0000C172700E201E301E001E1012500D2011C
:1038E000D30127006608043A0130031D0030F100BF
:1038F0006608053A0130031D0030F0007108F0043D
:103900000319AF2C02302800DA001030DB00E2305F
:10391000DC000230DD000830DE00803128259831DF
:1039200064000D30FB002D30FC00D730FD00FD0B96
:10393000972CFC0B972CFB0B972C000000000230FF
:103940002800DA001030DB002930DC000330DD0015
:103950000830DE008031282598316400E22C2700F1
:103960006608003A0319DF2C01302800DA00DB0179
:103970002030DC000330DD000830DE0080312825F7
:10398000983164000D30FB002D30FC00D730FD0075
:10399000FD0BC82CFC0BC82CFB0BC82C0000000036
:1039A00001302800DA00DB01D930DC000230DD0014
:1039B0000830DE008031282598316400E22C220096
:1039C0000D178D1710302500D6002730D700103086
:1039D000D4002730D5000020080090315D269831B2
:1039E00025004C08643A0319082DCC0A80302700C2
:1039F0005F06F000803061067002031D012D600833
:103A00005E020318072D6008DE006108DF00202D2C
:103A10002500CC0127005E082800B70027005F08BA
:103A20002800B800270062082800B90027006308B2
:103A30002800BA009031AC2098312700DE01DF0168
:103A4000270080306106F20080305D067202031D9F
:103A50002B2D5C086002013003180030F20080302A
:103A60005B06F100803061067102031D392D60088C
:103A70005A02013003180030F1008030F00080302D
:103A80005B067002031D462D5A08003C01300318E6
:103A90000030F0007108F0057208F0040319B42D2D
:103AA000640090315D26983125004C08643A031972
:103AB0006C2DCC0A803027005F06F0008030610654
:103AC0007002031D652D60085E0203186B2D6008EF
:103AD000DE006108DF00842D2500CC0127005E0890
:103AE0002800B70027005F082800B80027006208F8
:103AF0002800B900270063082800BA009031AC20E4
:103B000098312700DE01DF010D302800D30000309E
:103B1000D400D5010530D6000130D7008031FA2617
:103B2000983170080319972D01302500CA0025002F
:103B30004A08013A0130031D00302800AE000D3064
:103B4000D3000030D400D5010530D600D701803134
:103B5000FA2698312E08F0050319B32D3E242700CC
:103B6000E201E301B42D202D080003302800AD0050
:103B70002500CF012800B7019031682098312D0829
:103B80002500C800ED24003027006306031DCA2D60
:103B900000306206031DCD2D7D2E1430F400003060
:103BA000F5006208F0006308F100903100209831C0
:103BB0007008270062072800AB0071082700633DEA
:103BC0002800AC002D08AA0028002A081F3C031C6E
:103BD000762E2A08F00025004908F4008031BB2029
:103BE000983170082800B700903168209831ED2492
:103BF000003027006306031DFF2D00306206031D01
:103C0000022E7D2E80306306F000803028002C06C6
:103C10007002031D0E2E2B08270062020318742E5B
:103C200027001430F4000030F5006208F00063084B
:103C3000F1009031002098317008270062072800B9
:103C4000AB0071082700633D2800AC002A08F00093
:103C500025004908F4008031BB2098317008250008
:103C6000CF0028002D082500C800803027006306FB
:103C7000F00080307002031D3F2E7830620203187E
:103C8000422E762E28002D082A07F2007208AA007C
:103C900025004B08003A0130031D0030F100720886
:103CA000093A0130031D0030F0007108F0050319D6
:103CB0005D2E08302800AA00732E25004B08003A1C
:103CC0000130031D0030F10028002A08113A0130AC
:103CD000031D0030F0007108F0050319732E103039
:103CE000AA000430AD00752E762EE42D25004F0875
:103CF0002800B70090316820983108002500470857
:103D0000F0004608F4008031BB209831700828008C
:103D1000A400700825005007F40074082800A600CD
:103D20000530F20025004608F000F1017208031981
:103D30009D2EF035F10DFF3E972E01307002F200FE
:103D40000030713BF30080307306F0008030700269
:103D5000031DAC2E740872020318BA2E0530F00051
:103D600046082800A60070080319B92EA635FF3EA4
:103D7000B42EA60325005008280024020318C62EDE
:103D80002408250050022800A700C72EA7012708F5
:103D90002500D00028002708B70088312C2798314B
:103DA000ED24003027006306031DD82E0030620684
:103DB000031DDB2E632F62082800A800270063087C
:103DC0002800A9002500460828002707A500250887
:103DD0002602031C5C2F2508B70088312C27983158
:103DE000ED24003027006306031DF82E0030620624
:103DF000031DFB2E632F80306306F0008030280007
:103E000029067002031D072F280827006202031CE1
:103E1000142F3430FC00F130FD00FD0B0D2FFC0B96
:103E20000D2F00000000ED24803027006306F00015
:103E30008030280029067002031D212F2808270042
:103E40006202031C2E2F3430FC00F130FD00FD0B0C
:103E5000272FFC0B272F00000000ED2480302700C7
:103E60006306F0008030280029067002031D3B2FF6
:103E70002808270062020318562F2700620828002E
:103E8000A800270063082800A90025082500D00005
:103E9000803027006306F00080307002031D522F2F
:103EA000783062020318552F5C2F572F5C2F2500A6
:103EB00046082800A507E72E250050082800B7006F
:103EC00088312C27983108002000F8010830FC00C8
:103ED000700DF80D7408F8020318702FF80703101E
:103EE000F00DFC0B682F080027006C08F000F0367E
:103EF000F036F036F0360A30F4008031BB209831CD
:103F00000F3027006C05F1007108F007080027004A
:103F10004C08013C0318932FAE302800D3008831A1
:103F2000CD259831A42F27004C08013A031DA42F5A
:103F3000CF01CE012800E40180318D229831280084
:103F4000E40180318D22983108002700EB016A08D6
:103F5000093C0318C42F0A30F4006A08F0006427F3
:103F600070082700EB007008EB00EB35EB35EB3504
:103F7000EB350A30F4006A08F00064277808F00096
:103F800070082700EB04C62F6A08EB006B08F000EE
:103F90000800640021009712171697111715971043
:103FA000640023008C010C148C148D0122009113E9
:103FB000931378302100990020008C018D018E012F
:103FC000403022008C008D018E01033021008C00D6
:103FD00007308D008E018031F12798311E149E1418
:103FE000951324000D148D140D158B130800120069
:103FF0001E00F003031DF72FF103031DF72F080028
:1040000025004808F0004908F4008031BB20A031A9
:1040100070082800A400700825004F07F4007408F9
:104020002800A6000530F20025004908F000F10143
:10403000720803191F28F035F10DFF3E19280130D1
:104040007002F2000030713BF30080307306F00024
:1040500080307002031D2E287408720203183C2859
:104060000530F00049082800A600700803193B2815
:10407000A635FF3E3628A60325004F082800240257
:1040800003184828240825004F022800A7004928C3
:10409000A70127082500CF0028002708B700903186
:1040A0006820A0319831ED24A0310030270063064C
:1040B000031D5C2800306206031D5F28ED2862089E
:1040C0002800A800270063082800A9002500490847
:1040D00028002707A50025082602031CE628250836
:1040E000B70090316820A0319831ED24A031003024
:1040F00027006306031D7E2800306206031D812809
:10410000ED2880306306F000803028002906700218
:10411000031D8D28280827006202031C9C283430C8
:10412000FC00F130FD00FD0B9328FC0B93280000F0
:1041300000009831ED24A031803027006306F000A4
:104140008030280029067002031DA92828082700AE
:104150006202031CB8283430FC00F130FD00FD0B76
:10416000AF28FC0BAF28000000009831ED24A031EF
:10417000803027006306F000803028002906700296
:10418000031DC5282808270062020318E02827001D
:1041900062082800A800270063082800A900250855
:1041A0002500CF00803027006306F00080307002C9
:1041B000031DDC28783062020318DF28E628E12896
:1041C000E628250049082800A5076B2825004F0888
:1041D0002800B70090316820A03108000330280083
:1041E000A900A50129082500C70003302800A60062
:1041F0001430F4000030F50027006208F000630876
:10420000F10090310020A0317008270062072800DB
:10421000A70071082700633D2800A800A40128001A
:1042200024081F3C031CAB292408F0002500460885
:10423000F4008031BB20A03170082800B70088311D
:104240002C27A0319831B525A0319831ED24A0312B
:10425000003027006306031D2F2900306206031D6E
:104260003229C92980306306F000803028002806F2
:104270007002031D3E292708270062020318A9299E
:1042800027001430F4000030F5006208F0006308E5
:10429000F10090310020A03170082700620728004B
:1042A000A70071082700633D2800A8002408F0003B
:1042B00025004608F4008031BB20A031700825009D
:1042C000D0004F082800A50029082500C70048088D
:1042D0002800A600803027006306F00080307002BE
:1042E000031D74297830620203187729AB2928004E
:1042F00029082407F2007208A40025004D08003A9E
:104300000130031D0030F1007208093A0130031D2D
:104310000030F0007108F0050319922908302800D8
:10432000A400A82925004D08003A0130031D0030E3
:10433000F10028002408113A0130031D0030F0007C
:104340007108F0050319A8291030A4000430A90051
:10435000AA29AB290F29280025082500CF005008DD
:104360002800B70088312C27A03125004F082800ED
:10437000B70090316820A03126082500C8003430ED
:10438000FC00F130FD00FD0BC329FC0BC32900002C
:104390000000080027006208EE006308EF00EE202E
:1043A000003027006306031DD72900306206031D75
:1043B000DD2998312324A031302B9831ED24A03110
:1043C000803027006306F00080307002031DEA2968
:1043D000783062020318ED29302B98317E26A03107
:1043E000003027006306031DF72900306206031D15
:1043F000FD2998312324A031302B9831ED24A031B0
:10440000803027006306F00080307002031D0A2A06
:104410007830620203180D2A302B0020003027006C
:104420006306031D152A00306206031D1B2A9831FE
:104430002324A031302B9831ED24A0318030270087
:104440006306F00080307002031D282A7830620273
:1044500003182B2A302B80306306F1008030710264
:10446000031D342AC8306202013003180030F10005
:1044700080306306F00080306F067002031D422A10
:104480006E086202013003180030F00070087105F8
:10449000F30062086E02F10063086F3BF2008030A7
:1044A000F000803072067002031D582A7108643CC7
:1044B000013003180030F0007308F0050319612A79
:1044C000302B6208EE006308EF002500500828003A
:1044D000A000A10125004F082800A200A30125008B
:1044E0005108013A031D762AD101782A0130D10002
:1044F00098312324A031250051082800B7008831C5
:104500001A27A0310230FB000430FC00BA30FD0055
:10451000FD0B882AFC0B882AFB0B882A00009831A7
:10452000ED24A031803027006306F0008030700257
:10453000031D9C2A7830620203189F2A302BEE203C
:10454000003027006306031DA72A00306206031D02
:10455000AD2A98312324A031302B9831ED24A0319D
:10456000803027006306F00080307002031DBA2AF5
:10457000783062020318BD2A302B98317E26A03194
:10458000003027006306031DC72A00306206031DA2
:10459000CD2A98312324A031302B9831ED24A0313D
:1045A000803027006306F00080307002031DDA2A95
:1045B000783062020318DD2A302B002000302700FB
:1045C0006306031DE52A00306206031DEB2A9831BD
:1045D0002324A031302B9831ED24A03180302700E6
:1045E0006306F00080307002031DF82A7830620202
:1045F0000318FB2A302B80306F06F00080306306F2
:104600007002031D052B62086E0203182F2B250074
:104610005108013A031D0E2BD101102B0130D1009E
:1046200051082800B70088311A27A031200825003A
:10463000D000280022082500CF0028002008B7005D
:1046400088312C27A03125004F082800B700903171
:104650006820A03127006E08E2006F08E3006400C4
:10466000080064002500CC012700DE01DF012500E1
:10467000CA019831ED24A031803027006306F00094
:1046800080307002031D462B6E3062020318492BE6
:104690001B2C98312324A03121004F08003A031D20
:1046A000542B88310020A0310230FB000430FC0084
:1046B000BA30FD00FD0B5A2BFC0B5A2BFB0B5A2B6F
:1046C00000009831ED24A03127006208B40063088F
:1046D000B50080306306F00080307002031D722B3D
:1046E0006E3062020318752B1B2C8030F100803075
:1046F00033067102031D7E2B32086E3C0130031815
:104700000030F10080303306F00080306306700224
:10471000031D8C2B62083202013003180030F000B8
:104720007108F0050319952B1B2CCA2100302700B6
:104730006306031D9D2B00306206031DA32B9831D9
:104740002324A0311B2C803027006306F00080302A
:104750007002031DAD2B783062020318B02B1B2CA6
:1047600021006D08053A0130031D0030F1006C088E
:10477000053A0130031D0030F0007108F0050319FF
:10478000C22B1B2C6C08053C0318CE2B25004608B9
:10479000C7000130C60098317E26A0318030270046
:1047A0006306F00080307002031DD82B783062025F
:1047B0000318DB2B1B2C21006D08053C0318E62B8E
:1047C00025004908C8000130C900002021006C08FC
:1047D000053A031DEF2B01302500C600002C2100F7
:1047E0006C08063A031DF82B02302500C600002C89
:1047F00021006C08073A031D002C04302500C60078
:1048000021006D08053A031D092C01302500C9005F
:104810001A2C21006D08063A031D122C02302500C7
:10482000C9001A2C21006D08073A031D1A2C043008
:104830002500C9006400080080313E20A031270017
:1048400045082900A30080310320A0312900A301DD
:1048500080310320A031AE302900A3008031032035
:10486000A03127004C08023A0130031D0030F1004E
:104870004C08033A0130031D0030F0007108F004C9
:104880000319F82CD5302900A30080310320A03172
:1048900080302900A30080310320A031A8302900F6
:1048A000A30080310320A0313F302900A3008031D4
:1048B0000320A031D3302900A30080310320A03190
:1048C00027004C08023A031D6C2C44082900A30061
:1048D00080310320A031742C270044081F3E29009A
:1048E000A30080310320A03140302900A300803193
:1048F0000320A0318D302900A30080310320A03196
:1049000014302900A30080310320A0318130290018
:10491000A30080310320A031B4302900A3008031EE
:104920000320A031D9302900A30080310320A03119
:1049300022302900A30080310320A031203029003B
:10494000A30080310320A03102302900A300803170
:104950000320A03121302900A30080310320A031A1
:104960002900A30180310320A0317F302900A3005A
:1049700080310320A0312E302900A3008031032094
:10498000A03127004C08023A031DD32CA030290087
:10499000A30080310320A031C0302900A300803162
:1049A0000320A031DF2CA1302900A3008031032097
:1049B000A031C8302900A30080310320A031DA30B3
:1049C0002900A30080310320A03102302900A30078
:1049D00080310320A031DB302900A3008031032087
:1049E000A03140302900A30080310320A031A02D48
:1049F000D5302900A30080310320A0318030290068
:104A0000A30080310320A031A8302900A300803109
:104A10000320A0313F302900A30080310320A031C2
:104A2000D3302900A30080310320A031270044089F
:104A30002900A30080310320A03140302900A300C9
:104A400080310320A0318D302900A3008031032064
:104A5000A03114302900A30080310320A03181301F
:104A60002900A30080310320A031FF302900A300DA
:104A700080310320A031D9302900A30080310320E8
:104A8000A031F1302900A30080310320A031203073
:104A90002900A30080310320A03102302900A300A7
:104AA00080310320A03121302900A3008031032070
:104AB000A0312900A30180310320A0317F302900DB
:104AC000A30080310320A0312E302900A3008031C3
:104AD0000320A03127004C08043A031D7C2DA03090
:104AE0002900A30080310320A031C0302900A30099
:104AF00080310320A031882DA1302900A30080310E
:104B00000320A031C8302900A30080310320A03148
:104B1000DA302900A30080310320A03112302900AF
:104B2000A30080310320A031DB302900A3008031B5
:104B30000320A03140302900A30080310320A031A0
:104B4000A4302900A30080310320A031A630290021
:104B5000A30080310320A0318031D320A031033065
:104B6000FB000830FC007730FD00FD0BB52DFC0B81
:104B7000B52DFB0BB52D80313E20A0312700450817
:104B80002900A30080310320A03140302900A30078
:104B900080310320A03127004C08023A0130031D68
:104BA0000030F1004C08033A0130031D0030F000E2
:104BB0007108F0040319FA2DED016D08033C031C84
:104BC000F92D6D082800EE00EF0180315D20A03145
:104BD0002700EC01270080306C020318F62DEC0A48
:104BE0002900A30180310320A031EA2D2700ED0A1E
:104BF000DD2D172EED016D08073C031C172E6D08E7
:104C00002800EE00EF0180315D20A0312700EC018B
:104C1000270080306C020318142EEC0A2900A3012F
:104C200080310320A031082E2700ED0AFB2D8031B2
:104C3000D320A031AF302800D3008831CD25A0315A
:104C40000800640027006608043A0130031D0030A4
:104C5000F1006608053A0130031D0030F0007108CC
:104C6000F0040319422E02302800DA004030DB0045
:104C7000A830DC000230DD000430DE008031282561
:104C8000A031592E27006608003A0319562E01302C
:104C90002800DA000430DB00EB30DC000130DD00FE
:104CA0000430DE0080312825A031592E22000D1756
:104CB0008D17312327006608003A031D822E8030AD
:104CC000F000803063067002031D682E6208963C77
:104CD000031C6E2E22000D138D17812E8030F000E4
:104CE0008030270063067002031D782E6208FA3CAC
:104CF000031C7E2E20000D138D13812E20000D1716
:104D00008D13972E25004E08003A0130031D003008
:104D1000F10021004F08003A0130031D0030F0007F
:104D20007108F0040319972E88310020A031FF305C
:104D30002800AF0025004F082800B0009831052456
:104D4000A031FE302800AF00250050082800B00038
:104D500098310524A031FD302800AF00250051080E
:104D60002800B00098310524A031FC302800AF00A5
:104D70000030F4000130F50027003408F000350859
:104D8000F10090310020A03170082800B000983167
:104D90000524A031FB302800AF000030F4000130C2
:104DA000F50027003408F0003508F10090310020AC
:104DB000A0317808F0007908F10070082800B000F0
:104DC00098310524A03110302500D6002730D700B7
:104DD0001030D4002730D50098310020A0312700B2
:104DE00062082500D200270063082500D3002200B6
:104DF0008C130C1764000800640027006608043A4E
:104E00000130031D0030F1006608053A0130031D32
:104E10000030F0007108F0040319622F20003F08F1
:104E2000003A031D142F64000430FB000C30FC001A
:104E30003330FD00FD0B1A2FFC0B1A2FFB0B1A2F22
:104E40000000000026003608013A031D352F280017
:104E5000DA011030DB003330DC000230DD000830D6
:104E6000DE0080312825A031422F2800DA011030E1
:104E7000DB002A30DC000230DD000830DE0080314B
:104E80002825A03102302800DA001030DB003C3049
:104E9000DC000230DD000830DE0080312825A03142
:104EA000260065080319612F2800DA017030DB0045
:104EB0005730DC000230DD000130DE008031282573
:104EC000A031B72F27006608003A0319B72F20003A
:104ED0003F08003A031D6D2F64000430FB000C30C6
:104EE000FC003330FD00FD0B732FFC0B732FFB0B0D
:104EF000732F0000000026003608013A031D8D2F95
:104F00002800DA01DB014E30DC000230DD00083021
:104F1000DE0080312825A031992F2800DA01DB013D
:104F20004530DC000230DD000830DE00803128250D
:104F3000A03101302800DA00DB01CE30DC00013086
:104F4000DD000830DE0080312825A031260065080C
:104F50000319B72F2800DA010830DB00EE30DC003F
:104F60000030DD000130DE0080312825A0316400F2
:104F700088310020A03108002700EC019031F5278E
:104F8000A03170082700C5000130EC009031F527F2
:104F9000A03170082700CC007008003A031DD72FFD
:104FA00021000D138D1322000D178D17DD2F210009
:104FB0000D178D1722000D138D1308002034203497
:104FC0002034203420342034203420342034003461
:104FD0005034573452343D3430342E343034573416
:104FE00000345034573452343D342034203430347B
:104FF00057340034013400340034003400340034B9
:1050000027006608043A0130031D0030F1006608ED
:10501000053A0130031D0030F0007108F004031957
:105020001F282800DA010A30DB00C430DC00013020
:10503000DD000930DE0080312825A8313128270025
:105040006608003A031931282800DA010330DB0032
:10505000D730DC000130DD000930DE00803128254A
:10506000A83164000B30FB002630FC005D30FD00F1
:10507000FD0B3828FC0B3828FB0B382800000000FB
:1050800064000B30FB002630FC005D30FD00FD0BA2
:105090004728FC0B4728FB0B472800000000640052
:1050A0000B30FB002630FC005D30FD00FD0B562868
:1050B000FC0B5628FB0B56280000000064000B3048
:1050C000FB002630FC005D30FD00FD0B6528FC0B6D
:1050D0006528FB0B652800000000640027006608B7
:1050E000043A0130031D0030F1006608053A013032
:1050F000031D0030F0007108F00403198D2828000A
:10510000DA010A30DB002030DC000230DD0009303B
:10511000DE0080312825A8319F2827006608003A44
:1051200003199F282800DA010330DB00E130DC009E
:105130000130DD000930DE0080312825A8319831AA
:105140002324A83101302500D10001302800B70008
:1051500088311A27A831FF30AF0025004F082800FA
:10516000B00098310524A831FE302800AF0025009A
:1051700050082800B00098310524A831FD302800DF
:10518000AF00250051082800B00098310524A8314F
:1051900027006608043A0130031D0030F10066085C
:1051A000053A0130031D0030F0007108F0040319C6
:1051B000E7282800DA017030DB006E30DC000130B7
:1051C000DD000130DE0080312825A831F9282700D4
:1051D0006608003A0319F9282800DA010830DB00D4
:1051E0005930DC000230DD000130DE00803128253E
:1051F000A83101302000BF00A031FC26A8310800F2
:1052000007302700EC009031F527A83170082700FF
:10521000C4000830EC009031F527A8317008270051
:10522000C7004C08013C03181929A0311C24A831DF
:105230008C2927004C08013A031D8C290130CF002E
:10524000CE0103302800E40080318D22A8311A30CD
:10525000FC00F830FD00FD0B2B29FC0B2B29000076
:1052600003302800E40080318D22A8310630FC0094
:105270003030FD00FD0B3A29FC0B3A2900000330C9
:105280002800E40080318D22A83102302800E4009B
:1052900080318D22A83102302800E40080318D2237
:1052A000A83108302800E40080318D22A831280080
:1052B000E40180318D22A83108302800E4008031DB
:1052C0008D22A8312800E40180318D22A8310130DF
:1052D0002800E40080318D22A8311A30FC00F8301B
:1052E000FD00FD0B7129FC0B712900002800E40171
:1052F00080318D22A83106302800E40080318D22D3
:10530000A8312800E40180318D22A8310C3028001A
:10531000E40080318D22A831080026006F082800A3
:10532000DA00DB01BD30DC000330DD0080315323C7
:10533000A8310A3026006F02031CA2292700410869
:10534000B600A52927003030B6002E30B70042083D
:10535000B8006608043A0130031D0030F100660809
:10536000053A0130031D0030F0007108F004031904
:10537000C82904302800DA000630DB00B630DC0033
:105380000330DD000330DE0080312825A831DA2922
:1053900027006608003A0319DA2901302800DA00EC
:1053A000DB01B630DC000330DD000330DE0080318D
:1053B0002825A83108000D302800D3000030D40083
:1053C000D5013230D600D7018031FA26A8317008D5
:1053D0000319932A0630FB001330FC00AD30FD00AA
:1053E000FD0BF029FC0BF029FB0BF029000000005D
:1053F000640020000D1C0F2A25005108003A031DEF
:10540000042A0130D100052AD10151082800B70033
:1054100088311A27A83188310020A8317F2A260038
:105420006A08013A031D162AEA01182A0130EA0027
:105430006A08013A031D4E2A27006608043A013023
:10544000031D0030F1006608053A0130031D0030ED
:10545000F0007108F00403193B2A2800DA017030CB
:10546000DB006830DC000330DD000130DE0080311D
:105470002825A8314D2A27006608003A03194D2A2D
:105480002800DA010830DB006B30DC000330DD007F
:105490000130DE0080312825A8317F2A27006608E8
:1054A000043A0130031D0030F1006608053A01306E
:1054B000031D0030F0007108F00403196D2A280064
:1054C000DA017030DB006630DC000330DD000130D3
:1054D000DE0080312825A8317F2A27006608003A9F
:1054E00003197F2A2800DA010830DB003330DC00A2
:1054F0000330DD000130DE0080312825A8310D3079
:105500002800D3000030D400D5013230D600D701B6
:105510008031FA26A83170080319932A98310020A7
:10552000A83164007F2A0D302800D3000030D40059
:105530000230D5003230D600D7018031FA26A831AA
:1055400070080319192B640020000D19192B053060
:10555000F20025004608F000F10172080319B42A90
:10556000F035F10DFF3EAE2A01307002F20000303E
:10557000713BF3008030F000803073067002031D31
:10558000C42A250072085002013003180030F000D0
:1055900026006A08F0050319D62A2500D00A50080B
:1055A0002800B70088312C27A831092B26006A086B
:1055B0000130031D0030F4000530F20025004608DC
:1055C000F000F10172080319E92AF035F10DFF3EF0
:1055D000E32A01307002F2000030713BF3008030AA
:1055E000F000803073067002031DF92A250072084E
:1055F0004F02013003180030F0007408F005031961
:10560000092B2500CF0A4F082800B70090316820E9
:10561000A83188310020A83198310020A8319C3071
:10562000FC00D730FD00FD0B132BFC0B132B64008B
:10563000A42A0D302800D3000030D4000130D5005A
:105640003230D600D7018031FA26A8312600320840
:10565000003A0130031D0030F1007108F005031914
:10566000722B640020008D18722B25005008003C1E
:10567000013003180030F00026006A08F005031915
:105680004A2B2500D00350082800B70088312C276A
:10569000A831622B26006A080130031D0030F1009A
:1056A00025004F08003C013003180030F00071085D
:1056B000F0050319622BCF034F082800B700903183
:1056C0006820A83188310020A83198310020A83105
:1056D0009C30FC00D730FD00FD0B6C2BFC0B6C2BC1
:1056E0006400322B080027006918782B7414792B7A
:1056F00074100D302800D3000030D400D5013230B2
:10570000D6000130D7008031FA26A831F101741893
:10571000F10A7108F00503198F2B2700691427007F
:105720006918942B7414952B74100D302800D30035
:105730000030D400D5013230D600D7018031FA26AE
:10574000A831F1017418F10A7108F0050319C22B90
:1057500025006D08F0008031E227A83126003808C6
:10576000F4003908F5003A08F6003B08F7008031EC
:105770006127A8318831A222A83170082500EE00E7
:105780007108EF000D302800D3000030D400D5019F
:105790003230D600D7018031FA26A831F101270036
:1057A0006918F10A7108F00526006408F00403196D
:1057B000722C25006B08003A031D172C6C08013A67
:1057C000031DF62B50082800B70088312C27A8317C
:1057D00025004F082800B70090316820A831250027
:1057E00051082800B70088311A27A8310130250058
:1057F000EB008831AC27A83125006D08F00080311E
:10580000E227A83126003808F4003908F5003A08E4
:10581000F6003B08F70080316127A8318831A222C9
:10582000A83170082500EE007108EF001A2F6D08EE
:10583000F0008031E227A83126003808F40039084A
:10584000F5003A08F6003B08F70080316127A831DF
:105850008831A222A83170082500EE007108EF00FF
:105860000630FB001330FC00AD30FD00FD0B362C84
:10587000FC0B362CFB0B362C0000000064002600CD
:105880006408003A0130031D0030F10020000D18BB
:105890004B2C03104C2C0314F0010318F00A710870
:1058A000F0050319592C98313E24A8312600B20185
:1058B000722C22008C170C130630FB001330FC00F6
:1058C000AD30FD00FD0B622CFC0B622CFB0B622C3F
:1058D00000000000A0312126A8312600B201E40119
:1058E000270069100D302800D3000030D4000230AA
:1058F000D5003230D600D7018031FA26A8317008A1
:105900000319F02D25006B08003A031DC02C6C080C
:10591000013A031D9F2C50082800B70088312C271E
:10592000A83125004F082800B70090316820A83121
:10593000250051082800B70088311A27A831013006
:105940002500EB008831AC27A83125006D08F00058
:105950008031E227A83126003808F4003908F50024
:105960003A08F6003B08F70080316127A8318831FA
:10597000A222A83170082500EE007108EF001A2F4E
:105980006D08F0008031E227A83126003808F400C5
:105990003908F5003A08F6003B08F7008031612726
:1059A000A8318831A222A83170082500EE007108C4
:1059B000EF00640026003208003A031D1B2D013061
:1059C000B20025004F082400E800250050082400FC
:1059D000E700250051082400E6002500CF01580803
:1059E0000319F52CFF30D000F62CD0010130D10086
:1059F00050082800B70088312C27A83125004F080F
:105A00002800B70090316820A831250051082800EF
:105A1000B70088311A27A83125004E08003A031D27
:105A2000142D88310020A831260065082400EF00DD
:105A30002600E501492DB201240068082500CF00A9
:105A4000240067082500D000240066082500D10046
:105A5000240068082800B70090316820A83125008C
:105A600050082800B70088312C27A831250051089C
:105A70002800B70088311A27A83125004E08003ABF
:105A8000031D452D88310020A83124006F08260011
:105A9000E50027006608043A0130031D0030F100DC
:105AA0006608053A0130031D0030F0007108F0046B
:105AB0000319982D260032080130031D0030F00034
:105AC0006508F0050319722D2800DA017030DB003B
:105AD000B330DC000230DD000130DE0080312825EB
:105AE000A831972D260065080130031D0030F00015
:105AF0003208F00503198A2D2800DA017030DB0026
:105B0000B130DC000230DD000130DE0080312825BC
:105B1000A831972D2800DA017030DB00B530DC00A9
:105B20000230DD000130DE0080312825A831DA2D79
:105B300027006608003A0319DA2D260032080130E2
:105B4000031D0030F0006508F0050319B52D28008D
:105B5000DA010830DB00BB30DC000230DD00013050
:105B6000DE0080312825A831DA2D260065080130B5
:105B7000031D0030F0003208F0050319CD2D280078
:105B8000DA010830DB00B930DC000230DD00013022
:105B9000DE0080312825A831DA2D2800DA0108300E
:105BA000DB00B730DC000230DD000130DE00803188
:105BB0002825A83164000D302800D3000030D4001F
:105BC0000230D5003230D600D7018031FA26A83114
:105BD00070080319F02D98310020A8316400DB2DE6
:105BE0000D302800D3000030D4000130D500323011
:105BF000D600D7018031FA26A83126003208003AB3
:105C00000130031D0030F1007108F00503191A2F4F
:105C100025006B08003A031D462E6C08013A031D4F
:105C2000252E50082800B70088312C27A8312500E0
:105C30004F082800B70090316820A831250051088E
:105C40002800B70088311A27A83101302500EB0061
:105C50008831AC27A83125006D08F0008031E2279B
:105C6000A83126003808F4003908F5003A08F60093
:105C70003B08F70080316127A8318831A222A83182
:105C800070082500EE007108EF001A2F6D08F00073
:105C90008031E227A83126003808F4003908F500E1
:105CA0003A08F6003B08F70080316127A8318831B7
:105CB000A222A83170082500EE007108EF006400F0
:105CC00026006508003A031D682E0130E500692EA4
:105CD000E50102302800AF00260065082800B0006A
:105CE00098310524A83127006608043A0130031DC5
:105CF0000030F1006608053A0130031D0030F00065
:105D00007108F0040319C22E260032080130031D69
:105D10000030F0006508F00503199C2E2800DA0118
:105D20007030DB00A430DC000230DD000130DE002A
:105D300080312825A831C12E260065080130031DB9
:105D40000030F0003208F0050319B42E2800DA0103
:105D50007030DB00A230DC000230DD000130DE00FC
:105D600080312825A831C12E2800DA017030DB00EF
:105D7000A030DC000230DD000130DE00803128255B
:105D8000A831042F27006608003A0319042F2600C3
:105D900032080130031D0030F0006508F0050319DA
:105DA000DF2E2800DA010830DB00A630DC000230EC
:105DB000DD000130DE0080312825A831042F2600C7
:105DC00065080130031D0030F0003208F0050319AA
:105DD000F72E2800DA010830DB00AF30DC0002309B
:105DE000DD000130DE0080312825A831042F280095
:105DF000DA010830DB00AD30DC000230DD000130BC
:105E0000DE0080312825A83164000D302800D30041
:105E10000030D4000130D5003230D600D7018031B7
:105E2000FA26A831700803191A2F98310020A831DA
:105E30006400052F0800203420342034203420341E
:105E400020342034203400344F3456344534523416
:105E50004C344F3441344434003420342034203422
:105E60002034203420342034203400344F3456344D
:105E7000453452344C344F3441344434003441348A
:105E80004E343D34203420343034573400344534DB
:105E9000463446343D342034203430342534003404
:105EA00041344E3454343D3430342E34303457344D
:105EB000003441344E343D3430342E343034573491
:105EC00000344534463446343D34203430342534AF
:105ED00000344634693464346534723420344C34CC
:105EE0006F3473347334203469346E3470347534E1
:105EF0007434003464344234003469346E347034A1
:105F00007534743400346434423400340034303432
:105F10002E3430343034003430342E343034303495
:105F200000340034463469346434653472342034C7
:105F30004C346F3473347334003446344134533446
:105F400054342034543445345334543400344634B7
:105F50004134533454342034543445345334543459
:105F600000347534483400344C343D34003400344B
:105F70006334003401340034203433343334133484
:105F80008034203420342034203420342034203411
:105F90002034003400344F345634453452344C34B9
:105FA0004F344134443400344F3456344534523441
:105FB0004C344F34413444340034203420342034C1
:105FC0002034203420342034203400340034003491
:105FD000003400340034633400346C340034013451
:105FE0006C340034203420342034203420342034E5
:105FF0002034203420340034003407340734FF3F89
:10600000640001302700EC009031F527B0317008B2
:106010002700E6000230EC009031F527B03170081F
:10602000013A031D162801302600E5000330270041
:10603000EC009031F527B03170082700EC00983162
:106040007427B0317008E400E5010430EC009031B1
:10605000F527B03170082700EC0098317427B03173
:106060000A30F4008031BB20B03170082700E7000F
:106070007108E8000530EC009031F527B031700868
:106080002700EC0098317427B0310A30F4008031D9
:10609000BB20B03170082700DC007108DD0006303D
:1060A000EC009031F527B03170082700EC009831F2
:1060B0007427B0310A30F4008031BB20B031700851
:1060C0002700DA007108DB000930EC009031F52779
:1060D000B03170082700EC0098317427B0310A30D5
:1060E000F4008031BB20B03170082700B200710885
:1060F000B3000A30EC009031F527B0317008210070
:10610000EC000B302700EC009031F527B03170081F
:106110002500CD000C302700EC009031F527B03180
:1061200070082100ED000D302700EC009031F527BC
:10613000B03170082500CB000E302700EC00903104
:10614000F527B03170082600B5000F302700EC00AD
:106150009031F527B03170082500D8006400103068
:106160002700EC009031F527B03170082700EC00D3
:1061700098317427B0316430F4008031BB20B031E5
:1061800070082700EA007108EB001130EC00903134
:10619000F527B03170082700EC0098317427B03132
:1061A00070086A072600ED00003027006B3D2600CE
:1061B000EE0012302700EC009031F527B031700866
:1061C0002700EC0098317427B0316430F40080313E
:1061D000BB20B03170082700EA007108EB001330D3
:1061E000EC009031F527B03170082700EC009831B1
:1061F0007427B03170086A07AA0000306B3DAB000D
:106200001430EC009031F527B03170082700EC0015
:1062100098317427B0316430F4008031BB20B03144
:1062200070082700EA007108EB001530EC0090318F
:10623000F527B03170082700EC0098317427B03191
:1062400070086A07A80000306B3DA9001630EC000A
:106250009031F527B03170082700EC009831742791
:10626000B0316430F4008031BB20B03170082700B9
:10627000EA007108EB001730EC009031F527B031DF
:1062800070082700EC0098317427B03170086A0755
:10629000A60000306B3DA7001830EC009031F527C8
:1062A000B03170082700EC0098317427B0316430A9
:1062B000F4008031BB20B03170082700EA0071087B
:1062C000EB001930EC009031F527B0317008270051
:1062D000EC0098317427B03170086A07AC000030C8
:1062E0006B3DAD001A30EC009031F527B0317008ED
:1062F0002700EC0098317427B0316430F40080310D
:10630000BB20B03170082700EA007108EB001B3099
:10631000EC009031F527B03170082700EC0098317F
:106320007427B03170086A07B00000306B3DB100CF
:106330001C30EC009031F527B03170082700EC00DC
:1063400098317427B0316430F4008031BB20B03113
:1063500070082700EA007108EB001D30EC00903156
:10636000F527B03170082700EC0098317427B03160
:1063700070086A07AE0000306B3DAF002030EC00C3
:106380009031F527B03170082700EC009831742760
:10639000B0316430F4008031BB20B0317008270088
:1063A000EA007108EB002130EC009031F527B031A4
:1063B00070082700EC0098317427B03170086A0724
:1063C000A40000306B3DA5002230EC009031F52791
:1063D000B03170082700EC0098317427B031643078
:1063E000F4008031BB20B03170082700EA0071084A
:1063F000EB002330EC009031F527B0317008270016
:10640000EC0098317427B03170086A07A2000030A0
:106410006B3DA3002430EC009031F527B0317008BB
:106420002700EC0098317427B0316430F4008031DB
:10643000BB20B03170082700EA007108EB0025305E
:10644000EC009031F527B03170082700EC0098314E
:106450007427B03170086A07D40000306B3DD50056
:106460002630EC009031F527B03170082700EC00A1
:1064700098317427B0316430F4008031BB20B031E2
:1064800070082700EA007108EB002730EC0090311B
:10649000F527B03170082700EC0098317427B0312F
:1064A00070086A07D20000306B3DD3002830EC0042
:1064B0009031F527B03170082700EC00983174272F
:1064C000B0316430F4008031BB20B0317008270057
:1064D000EA007108EB002930EC009031F527B0316B
:1064E00070082700EC0098317427B03170086A07F3
:1064F000D00000306B3DD1002A30EC009031F52700
:10650000B03170082700EC0098317427B031643046
:10651000F4008031BB20B03170082700EA00710818
:10652000EB002B30EC009031F527B03170082700DC
:10653000EC0098317427B03170086A07D60000303B
:106540006B3DD7002C30EC009031F527B03170084E
:106550002700EC0098317427B0316430F4008031AA
:10656000BB20B03170082700EA007108EB002D3025
:10657000EC009031F527B03170082700EC0098311D
:106580007427B03170086A07D80000306B3DD9001D
:106590003030EC009031F527B03170082600B6009D
:1065A00031302700EC009031F527B031700827001A
:1065B000EC0098317427B03170082600B7003230F3
:1065C0002700EC009031F527B03170082700EC006F
:1065D00098317427B03170082500ED003330270062
:1065E000EC009031F527B03170082100CF00343035
:1065F0002700EC009031F527B03170082700EC003F
:1066000098317427B03170082600EF00353027002C
:10661000EC009031F527B03170082700EC0098317C
:106620007427B03170082500EC0064000800B83110
:106630001C21B031031A1F2B01302000CA009831F1
:10664000C927B0310730FB001730FC006A30FD006D
:10665000FD0B282BFC0B282BFB0B282B00006400C8
:106660000020A031BC27B03127006608003A031D86
:106670003C2B22000D178D1725006D08F00080318E
:10668000E227B03126003808F4003908F5003A084E
:10669000F6003B08F70080316127B0318831A22233
:1066A000B03170082500EE007108EF000730FB00E4
:1066B0001730FC006A30FD00FD0B5C2BFC0B5C2BE3
:1066C000FB0B5C2B0000640020008D18692B7414F8
:1066D0006A2B74100D196E2B03146F2B0310741C8E
:1066E000752B031C752B7414762B7410741C7D2B66
:1066F00001302100EB002600E50121006C08053A7D
:10670000031D862B01302500C600972B21006C0845
:10671000063A031D8F2B02302500C600972B21005F
:106720006C08073A031D972B04302500C600210092
:106730006D08053A031DA02B01302500C900B12BBF
:1067400021006D08063A031DA92B02302500C9005F
:10675000B12B21006D08073A031DB12B0430250031
:10676000C9000730FB001730FC006A30FD00FD0B4C
:10677000B72BFC0BB72BFB0BB72B000064000730CB
:10678000FB001730FC006A30FD00FD0BC52BFC0B35
:10679000C52BFB0BC52B000064000730FB00173036
:1067A000FC006A30FD00FD0BD32BFC0BD32BFB0B45
:1067B000D32B000064000730FB001730FC006A3068
:1067C000FD00FD0BE12BFC0BE12BFB0BE12B000093
:1067D00064000730FB001730FC006A30FD00FD0B41
:1067E000EF2BFC0BEF2BFB0BEF2B00006400A83111
:1067F0000021B03120008D18FF2B7414002C741070
:106800000D19042C0314052C0310741C0B2C031CF1
:106810000B2C74140C2C741020000D18112C031464
:10682000122C0310741C182C031C182C7414192C13
:106830007410741C792C27006608043A0130031D7B
:106840000030F1006608053A0130031D0030F00009
:106850007108F00403193A2C2800DA010C30DB002F
:106860006030DC000030DD000930DE00803128259A
:10687000B0314C2C27006608003A03194C2C280034
:10688000DA010330DB005630DC000030DD00093077
:10689000DE0080312825B031FF302800B70090316C
:1068A0006820B03125005808003A031D5E2CFF30E7
:1068B0002800B70088312C27B031632C2800B7019D
:1068C00088312C27B0310130B70088311A27B03118
:1068D00064000B30FB002630FC005D30FD00FD0B3A
:1068E0006F2CFC0B6F2CFB0B6F2C00000000640066
:1068F000692C280064000D30D3000030D400D5018D
:106900006430D600D7018031FA26B03170080319FF
:106910006A2D27006608043A0130031D0030F1009B
:106920006608053A0130031D0030F0007108F004DC
:106930000319C42C2800DA010630DB004B30DC00E0
:106940000030DD000A30DE0080312825B031023011
:106950002800DA000630DB003630DC000030DD00D5
:106960000530DE0080312825B03104302800DA00FF
:106970002A30DB003330DC000030DD000230DE0086
:1069800080312825B031E32C27006608003A03192E
:10699000E32C2800DA01DB012230DC000030DD00CE
:1069A0001030DE0080312825B03101302800DA00B7
:1069B0000330DB003C30DC000030DD000230DE0064
:1069C00080312825B03134302700EC009031F52794
:1069D000B03170082700EC0098317427B03170088E
:1069E0002600EF00A8318D21B0310D302800D300F2
:1069F0000030D4000230D5003230D600D7018031CB
:106A0000FA26B031700803192F2D633026006F026B
:106A100003181D2DEF0AA8318D21B03126006F0813
:106A20002700EA009831A527B03170082800B0008F
:106A30003430AF0098310524B0310D302800D30038
:106A40000030D4000230D5003230D600D70180317A
:106A5000FA26B031700803192F2D64001D2D0D305A
:106A6000D3000030D4000130D5003230D600D70139
:106A70008031FA26B03170080319682D26006F089E
:106A8000003C0318562DEF03A8318D21B0312600AC
:106A90006F082700EA009831A527B0317008280058
:106AA000B0003430AF0098310524B0310D302800EB
:106AB000D3000030D4000130D5003230D600D701E9
:106AC0008031FA26B03170080319682D6400562D04
:106AD0006400F52C21006B08003A031DBE2DFF3029
:106AE0002700EC009031F527B03170082500CF0069
:106AF000FE302700EC009031F527B03170082500FA
:106B0000D000FD302700EC009031F527B03170083F
:106B10002500D100FC302700EC009031F527B03182
:106B200070082700B500B401FB30EC009031F52768
:106B3000B03170082700B4070030B53D250050087B
:106B40002800B70088312C27B03125004F082800D5
:106B5000B70090316820B031250051082800B700F7
:106B600088311A27B03120004A08013A031DBA2D96
:106B70000130BF00A031FC26B031C12DA83100206A
:106B8000B03188310020B031270069146400983199
:106B90000020B03121006B08003A031DD32DA8312D
:106BA0007323B031D62DA831DB21B0310030250060
:106BB0006F06031DDD2D00306E060319E42D013034
:106BC000EE020030EF3B132E21006B08003A01303B
:106BD000031D0030F10025006D08003A0130031953
:106BE0000030F0007008F1056B08013A0130031D18
:106BF0000030F0007108F0050319132E6C0803191A
:106C00000E2E2800B70188312C27B031B701903102
:106C10006820B031B70188311A27B0312500EB0167
:106C200098318727B031C62D142EFF3F0034003431
:106C3000003400340034003400345F340034003455
:106C40000034073400340734003414347F341434EF
:106C50007F34143424342A347F342A3412342334D5
:106C600013340834643462343634493455342234AD
:106C700050340034053403340034003400341C3400
:106C80002234413400340034413422341C34003482
:106C900008342A341C342A340834083408343E3486
:106CA00008340834003450343034003400340834AC
:106CB00008340834083408340034303430340034B4
:106CC0000034203410340834043402343E34513457
:106CD000493445343E34003442347F344034003447
:106CE00042346134513449344634213441344534DA
:106CF0004B3431341834143412347F341034273484
:106D000045344534453439343C344A3449344934C3
:106D100030340134713409340534033436344934A1
:106D200049344934363406344934493429341E341C
:106D300000343634363400340034003456343634BB
:106D40000034003400340834143422344134143410
:106D500014341434143414344134223414340834C4
:106D600000340234013451340934063432344934A5
:106D7000793441343E347E341134113411347E344C
:106D80007F3449344934493436343E344134413413
:106D9000413422347F344134413422341C347F3432
:106DA00049344934493441347F3409340934013495
:106DB00001343E3441344134513432347F34083468
:106DC000083408347F34003441347F344134003493
:106DD0002034403441343F3401347F340834143497
:106DE000223441347F3440344034403440347F34A2
:106DF0000234043402347F347F34043408341034D1
:106E00007F343E344134413441343E347F3409349C
:106E10000934093406343E344134513421345E346B
:106E20007F340934193429344634463449344934DA
:106E300049343134013401347F34013401343F3476
:106E40004034403440343F341F3420344034203404
:106E50001F347F342034183420347F3463341434A6
:106E6000083414346334033404347834043403347D
:106E700061345134493445344334003400347F3470
:106E80004134413402340434083410342034413461
:106E900041347F3400340034043402340134023489
:106EA00004344034403440344034403400340134FD
:106EB0000234043400342034543454345434783498
:106EC0007F344834443444343834383444344434DB
:106ED0004434203438344434443448347F343834EF
:106EE000543454345434183408347E34093401345E
:106EF000023408341434543454343C347F34083469
:106F0000043404347834003444347D344034003460
:106F10002034403444343D34003400347F34103461
:106F200028344434003441347F34403400347C34D9
:106F300004341834043478347C340834043404348D
:106F40007834383444344434443438347C3414345D
:106F500014341434083408341434143418347C349D
:106F60007C340834043404340834483454345434FD
:106F70005434203404343F344434403420343C34DA
:106F80004034403420347C341C34203440342034A9
:106F90001C343C344034303440343C3444342834A1
:106FA0001034283444340C345034503450343C348D
:106FB0004434643454344C34443400340834363467
:106FC00041340034003400347F3400340034003461
:106FD0004134363408340034083408342A341C343C
:106FE000083408341C342A34083408342E3400346D
:106FF000FF3FFF3FFF3FFF3FFF3FFF3FFF3FFF3FA1
:107000007534483400344C343D3400347534003425
:107010004C343D34003420342034203420342034A7
:1070200020342034203400344F3456344534523424
:107030004C344F3441344434003420342034203430
:107040002034203420342034203400345334573456
:1070500052343D3420342034203420340034003481
:107060005334573452343D342034203420342034C7
:107070000034203420342034203420342034203490
:10708000203400344F345634453452344C344F3469
:1070900041344434003420340034203400345F342C
:1070A00000342E3400342034203420342034203472
:1070B00020342034203400340134003400340134CE
:1070C0000034003400340034003400340034003420
:1070D000003400341034273410342734003453344F
:1070E000573452343D3430342E343034303400345C
:1070F000523445345334453454342034203420340D
:1071000000345334573452343D3430342E34303418
:10711000303400345034573452343D3430342E340B
:107120003034573400345034573452343D342034E2
:1071300020343034573400342E3400346C3400346E
:1071400043343D34003470344634003443343D34E9
:107150000034703400340034003400347034463469
:10716000003443343D34003441344E3454343D34DF
:107170002034203430345734003441344E345434C5
:107180003D342034203430345734003445344634D0
:1071900046343D34203420343034253400344134F6
:1071A0004E3454343D3430342E343034573400347B
:1071B000543445345334543420344D344F344434EF
:1071C00045340034203400345F3400342E3400342D
:1071D0002E340034543455344E3445340034203485
:1071E00000345F3400345F3400342E3400345334C0
:1071F000573452343D3430342E343034303400344B
:10720000543445345334543420344D344F3444349E
:1072100045340034523445345334453454342034E6
:107220002034203400345334573452343D34303415
:107230002E3430343034003469308400AF3085006F
:107240004E30F0000130F10022308600003087001F
:107250009831F727B83100308400B83085004B30C2
:10726000F0000130F100A030860000308700983136
:10727000F727B8311B308400AF3085004E30F00066
:107280000130F10020308600013087009831F72767
:10729000B831FC308400AF3085000330F00001309D
:1072A000F100EB308600003087009831F727B831C5
:1072B000B4308400B83085002E30F0000130F10089
:1072C000A0308600013087009831F727B831F630BA
:1072D0008400B73085000230F0000130F100EE305C
:1072E0008600003087009831F727B831F7308400E6
:1072F000B83085001330F0000130F100CE30860048
:10730000013087009831F727B831FE3084008F3084
:1073100085000230F0000130F1006E30860001304F
:1073200087009831F727B831F2308400AF308500FC
:107330000A30F0000130F100E130860001308700B2
:107340009831F727B831DE308400A73085001C3033
:10735000F0000130F10020308600023087009831C3
:10736000F727B831F93084008F3085000530F00000
:107370000130F100EB308600013087009831F727AB
:10738000B83181308400B83085003330F0000130EE
:10739000F1003C308600023087009831F727B83181
:1073A000E2308400B83085001530F0000130F10083
:1073B000A0308600023087009831F727B831FF30BF
:1073C0008400A73085000130F0000130F1006F30FB
:1073D0008600023087009831F727B8314B3084009F
:1073E000B83085003630F0000130F100B53086004D
:1073F000023087009831F727B8310A308400B9305D
:1074000085001230F0000130F1002030860003309A
:1074100087009831F727B831FA308400A73085000B
:107420000530F0000130F100EB30860002308700BB
:107430009831F727B831B7308400AF3085003B3042
:10744000F0000130F10032308600033087009831BF
:10745000F727B8310800FF3FFF3FFF3FFF3FFF3FE7
:10746000FF3FFF3FFF3FFF3FFF3FFF3FFF3FFF3F2C
:10747000FF3FFF3FFF3FFF3FFF3FFF3FFF3FFF3F1C
:10748000FF3FFF3FFF3FFF3FFF3FFF3FFF3FFF3F0C
:10749000FF3FFF3FFF3FFF3FFF3FFF3FFF3FFF3FFC
:020000040001F9
:10E000007E00010000002500130005005000010003
:10E0100002000000070001000700010001000000ED
:10E0200001000000020000000400000008000000E1
:10E03000160000003200000064000000FF00FF0036
:10E0400000001000000022000000400000008200DC
:10E05000010060000300200006004000FF00FF00F8
:10E06000000020000000010000000000FF00FF0091
:10E07000FF00FF00FF00FF00FF00FF00FF00FF00A8
:10E08000FF00FF00FF00FF00FF00FF00FF00FF0098
:10E09000FF00FF00FF00FF00FF00FF00FF00FF0088
:10E0A000FF00FF00FF00FF00FF00FF00FF00FF0078
:10E0B000FF00FF00FF00FF00FF00FF00FF00FF0068
:10E0C000FF00FF00FF00FF00FF00FF00FF00FF0058
:10E0D000FF00FF00FF00FF00FF00FF00FF00FF0048
:10E0E000FF00FF00FF00FF00FF00FF00FF00FF0038
:10E0F000FF00FF00FF00FF00FF00FF00FF00FF0028
:10E10000FF00FF00FF00FF00FF00FF00FF00FF0017
:10E11000FF00FF00FF00FF00FF00FF00FF00FF0007
:10E12000FF00FF00FF00FF00FF00FF00FF00FF00F7
:10E13000FF00FF00FF00FF00FF00FF00FF00FF00E7
:10E14000FF00FF00FF00FF00FF00FF00FF00FF00D7
:10E15000FF00FF00FF00FF00FF00FF00FF00FF00C7
:10E16000FF00FF00FF00FF00FF00FF00FF00FF00B7
:10E17000FF00FF00FF00FF00FF00FF00FF00FF00A7
:10E18000FF00FF00FF00FF00FF00FF00FF00FF0097
:10E19000FF00FF00FF00FF00FF00FF00FF00FF0087
:10E1A000FF00FF00FF00FF00FF00FF00FF00FF0077
:10E1B000FF00FF00FF00FF00FF00FF00FF00FF0067
:10E1C000FF00FF00FF00FF00FF00FF00FF00FF0057
:10E1D000FF00FF00FF00FF00FF00FF00FF00FF0047
:10E1E000FF00FF00FF00FF00FF00FF00FF00FF0037
:10E1F000FF00FF00FF000000000001000000000021
:020000040001F9
:04000E00C43FFF1AD2
:020000040001F9
:08000000FF3FFF3FFF3FFF3F00
:00000001FF
